:020000040800F2
:10000000D83E0020E1010008354400083F390008CF
:1000100011410008051300082558000800000000E1
:10002000000000000000000000000000490100087E
:1000300045130008000000008D010008094F00086A
:10004000FB010008FB010008FB010008FB010008A0
:10005000FB010008FB01000847130008FB01000832
:10006000FB010008FB010008FB0100080913000860
:10007000FB010008FB010008FB010008FB01000870
:10008000FB010008FB010008FB010008FB01000860
:10009000FB010008FB010008FB010008FB01000850
:1000A000FB010008A54F0008FB010008FB01000848
:1000B0003550000821510008FB010008FB01000831
:1000C000FB010008FB010008FB010008FB01000820
:1000D000FB01000881570008FB010008FB01000834
:1000E000FB010008FB010008FB010008FB01000800
:1000F000FB010008FB010008FB010008FB010008F0
:10010000FB010008FB0100080D520008FB0100087C
:10011000FB010008FB010008FB0100086952000810
:10012000FB010008FB010008FB010008FB010008BF
:10013000DFF810D000F03EFD004800477173000862
:10014000AFF30080D83E0020224B19680868B0E861
:10015000F00F80F30988BFF36F8F4FF0000080F33A
:1001600011884EF00D0E7047000000000648006830
:10017000006880F3088862B661B6BFF34F8FBFF3A3
:100180006F8F00DF00BF00BF08ED00E0EFF30980D4
:10019000BFF36F8F0F4B1A6820E9F00F106008B59E
:1001A0004FF0500080F31188BFF34F8FBFF36F8F74
:1001B00008F028FB4FF0000080F31188BDE80840EC
:1001C00019680868B0E8F00F80F30988BFF36F8FF3
:1001D000704700BF8C010020EFF3058070470000DE
:1001E0000648804706480047FEE7FEE7FEE7FEE7D1
:1001F000FEE7FEE7FEE7FEE7FEE7FEE7A14F0008A9
:1002000031010008202A04DB203A21FA02F0002103
:10021000704721FA02F3D040C2F120029140084316
:100220001946704740EA01039B0703D009E008C95B
:10023000121F08C0042AFAD203E011F8013B00F8AB
:10024000013B521EF9D27047D2B201E000F8012BF7
:10025000491EFBD270470022F6E710B513460A4646
:1002600004461946FFF7F0FF204610BDF0B480EABF
:100270000102D40F4200B2EB410F02D202460846FF
:1002800011464A0042D0C30DDDB2C1F3C752AD1AC8
:10029000202D35DAC1F3160141F4000204B15242B7
:1002A000C5F1200602FA06F12A411044B3EBD05FF3
:1002B00023D0C4B1012DA0EBC35009DCF0BC4FF03A
:1002C000004202EAC352DBB200F5000000F096BA29
:1002D000400000F1807000EBC350A0F1807040EA54
:1002E000D170490009E0490841EAC071A0EBC35050
:1002F00000F50000400800EBC350F0BC00F075BAF8
:100300006142012202EB4101001BF6E7F0BC70479D
:1003100081F00041AAE780F00040A7E780EA0102EF
:1003200010B502F00043400022D04A001FD0010E59
:1003300001EB1261C0F35600C2F3560240F4000014
:1003400042F40002A0FB022000047F39140400D014
:10035000401C50EA124001D44000491EC2B20C06B3
:1003600004EBD010401C4008802A02D003E000209B
:1003700010BD20F00100002900DA0020184310BD54
:1003800030B480EA010202F0004530F0004221F072
:10039000004013D090B1C30DD40DC2F31601C0F3C9
:1003A0001600E41A41F4000140F400027D34914249
:1003B00001D3641C00E04900002C02DA30BC0020AC
:1003C00070474FF400000023914201D3891A034380
:1003D00040084FEA4101F7D151B1914202D14FF0AB
:1003E000004105E002D24FF0010101E06FF0010190
:1003F00003EBC450284430BC00F0F7B92DE9FE4FA0
:1004000081EA030404F0004421F0004100944FF01D
:10041000000B23F0004350EA01045ED052EA0304CB
:100420005BD0C3F30A54C1F30A552C44A4F2F3344D
:100430000194A0FB0254C1F3130141F48011C3F3F2
:10044000130343F4801301FB024400FB034E840AB0
:10045000970A44EA815447EA8357A4FB0768029548
:100460008D0A05FB07854FEA932C04FB0C542705E6
:10047000029D4FEA065847EA1637B5EB08056EEBC2
:10048000070C870E920E47EA811742EA8312A7FBF8
:100490000201B6EB0B0164EB00042B0D43EA0C33B5
:1004A0005E1844EB1C50DA465146E7FB0201C5F3E7
:1004B00013044FEA0B3343EA14534FEA0432019C0E
:1004C00043EA0603A4F10C040294009CCDE900B4B5
:1004D00000F0D1F903B0BDE8F08F00200146F9E744
:1004E0002DE9F04D81EA030404F0004B21F00045B2
:1004F00014464FF0000A23F0004150EA050220D0D4
:1005000054EA01021DD0C5F30A570246C5F313038E
:10051000C1F31300C1F30A5640F4801543F480136D
:10052000A7EB0608101BD64608F2FD3873EB050052
:1005300002D308F1010801E092185B41B8F1000F05
:1005400003DA00200146BDE8F08D00204FF4801151
:10055000064684460EE0171B73EB050705D3121BF6
:1005600063EB050306434CEA010C49084FEA3000EF
:1005700092185B4150EA0107EDD152EA030012D014
:1005800082EA040083EA0501084305D0101BAB4151
:1005900006D20122002306E000224FF0004302E0D1
:1005A0006FF0010253101AEB06004CEB085110EBF0
:1005B0000A0041EB0B01BDE8F04D00F04DB9C10F51
:1005C00080EAE0700844CA079623002100F016B9BB
:1005D00096230022114600F011B900F0004220F0ED
:1005E0000040C10DC0F3160040F400007F2901DA7D
:1005F00000207047962903DCC1F19601C84001E054
:1006000096398840002AF4D04042704720F00040DC
:10061000C10DC0F3160040F400007F2901DA00206C
:100620007047962903DCC1F19601C840704796399E
:100630008840704770B5C1F30A5201F000450024AC
:10064000C1F3130140F2FF3341F480119A4201DA01
:10065000002070BD40F233439A42A2F2334203DCE1
:100660005242FFF7CFFD00E090402C43F1D04042D2
:1006700070BDC1F30A5210B5C1F3130140F2FF334C
:1006800041F480119A4201DA002010BD40F2334358
:100690009A42A2F2334203DC5242FFF7B3FD10BD8F
:1006A000904010BD00F0004230F000400AD0C10D73
:1006B00001F56071C0F3160042EA0151C20840071B
:1006C00011437047002001467047000030B5041EFA
:1006D00071F1000404DB4FF00044404264EB01017F
:1006E000141E73F1000405DB1C464FF00043524218
:1006F00063EB04038B4208BF824230BD01F000432C
:1007000030B421F0004150EA010206D00A0DA2F5F2
:100710006072C1F31301002A02DC30BC0020704774
:10072000440F44EAC104C100E01830BC00EBC250E1
:1007300000F05BB8002801DBC0F10040002901DBBC
:10074000C1F1004181427047002801DBC0F1004047
:10075000002901DBC1F100418842704730B50B46EA
:10076000014600202022012409E021FA02F59D42E1
:1007700005D303FA02F5491B04FA02F52844151EB5
:10078000A2F10102F1DC30BD2DE9F05F0546002049
:1007900092469B4688460646814640241BE02846F2
:1007A000414647462246FFF72DFD53465A46C01A9A
:1007B000914110D311461846224600F00DFA2D1A29
:1007C00067EB01084F4622460120002100F004FAA1
:1007D00017EB00094E41201EA4F10104DFDC48465E
:1007E00031462A464346BDE8F09F0029A8BF70471E
:1007F000401C490008BF20F00100704710B4B0FA57
:1008000080FC00FA0CF050EA010404BF10BC7047F1
:1008100049B1CCF1200421FA04F411FA0CF118BF0B
:10082000012121430843A3EB0C01CB1D4FEA0061DA
:100830004FEA102042BF002010BC704700EBC350AD
:1008400010440029A4BF10BC7047401C490008BFD9
:1008500020F0010010BC704710B5141E73F10004A5
:1008600008DA401C41F1000192185B411A4301D1A2
:1008700020F0010010BD2DE9F04D92469B4611B1CC
:10088000B1FA81F202E0B0FA80F22032904600F034
:10089000A3F904460F4640EA0A0041EA0B01534619
:1008A0005A46084313D0114653EA010019D0C8F143
:1008B00040025046FFF7A6FC05460E4650465946F4
:1008C000424600F089F9084305D0012004E02046A3
:1008D0003946BDE8F08D0020054346EAE0762C431A
:1008E00037430A986305E40AA0EB08000022FD0ADA
:1008F00044EA47540A3002D500200146E9E70105E1
:1009000010196941DDE9084500196941BDE8F04D5C
:10091000A2E72DE9FE4F804681EA0300C00F0C4696
:10092000009021F0004123F00045B8EB0200A941FE
:1009300005D24046214690461C460B46024623F00F
:100940000040104347D0270DC7F30A00C3F30A51F4
:100950000290401A019040286BDAC3F3130040F470
:10096000801B0098924620B10023D2EB030A63EB70
:100970000B0B01985946C0F14002504600F02CF98B
:1009800006460D4650465946019A00F034F910EBE0
:1009900008006141002487EA115284EAE7731A4390
:1009A00040D0009A62B3019A012A4FEA075215DC3F
:1009B000001B61EB02014FF0004202EA0752CDE951
:1009C0000042001C41F5801132462B46FFF753FFD1
:1009D00003B0BDE8F08F40462146F9E7001B61EB0C
:1009E0000201001C41F5801300185B412018A2F59C
:1009F000001747EB030140EAD570B6196D4111E0CD
:100A00006D084FEA360645EAC0754FEA0752001BEB
:100A100061EB0201001C41F5801149084FEA3000EA
:100A20000019514132462B4603B0BDE8F04FFFF7A5
:100A300013BF0098012240000023D0EB020263EBB9
:100A4000E073009821464FEAE074B8EB000061EBD8
:100A50000401E9E783F000435BE781F0004158E7D8
:100A600070B521F0004303430CD0C1F30A550024B4
:100A7000D5EB040564EB0403D617AD1AB34102DBD2
:100A80000020014670BD201841EB025170BD2DE9D8
:100A9000F04D00231A461B1A8A4103DB0020014651
:100AA000BDE8F08DC1F30A52C1F3130141F4801582
:100AB0004FF0000BD10702D100186D41521E0027E4
:100AC000044640F2FF11384601EB620A3E4680467A
:100AD000024600204FF48011FFF794FBC2197141C8
:100AE000BB1846EB0100B4EB030C75EB000C04D310
:100AF000E41A65EB000517460E46241908F10100BB
:100B00006D4180463428E3DDF91946EB0600091BE8
:100B1000A84103D24FF0FF32134601E000221346F2
:100B20001BEB070046EB0A51BDE8F04DFFF794BE02
:100B30000EB5C10F80EAE0700844CA07002140F2F8
:100B400033438DE80E000A460B46FFF794FE03B0D0
:100B500000BDC1F30A52C1F3130140F2FF3341F467
:100B600080119A4202DA00200146704740F2334376
:100B70009A42A2F2334202DC5242FFF743BB00F03A
:100B80002BB8000030B5041E71F1000404DB4FF0F7
:100B90000044404264EB0101141E73F1000405DBC4
:100BA0001C464FF00043524263EB0403994208BFD6
:100BB000904230BD064C074D06E0E06840F001036E
:100BC00094E8070098471034AC42F6D3FFF7B4FA24
:100BD000A09C0008C09C0008202A04DB203A00FAF0
:100BE00002F1002070479140C2F1200320FA03F384
:100BF000194390407047202A06DBCB17203A41FA70
:100C000002F043EAE07306E041FA02F3D040C2F199
:100C10002002914008431946704770B58C1810F8AF
:100C2000015B15F0070301D110F8013B2A1106D131
:100C300010F8012B03E010F8016B01F8016B5B1E4B
:100C4000F9D12B0705D40023521E0DD401F8013B26
:100C5000FAE710F8013BCB1A921C03E013F8015B92
:100C600001F8015B521EF9D5A142D8D3002070BD16
:100C700070B5044600252068806800F0010018B3B4
:100C80002068806820F001002168886001F016FB70
:100C9000054613E001F012FB401B02280ED9206824
:100CA000806800F0010048B1A06A40F01000A06226
:100CB000E06A40F00100E062012070BD20688068B9
:100CC00000F001000028E5D10020F6E770B50546E8
:100CD0006C6AA06A00F05000E0B9A06A40F40070AD
:100CE000A0622068806800F46020B0F5602F0DD10C
:100CF000207B58B9A06A20F48070A062A06A00F43A
:100D0000805018B9A06A40F00100A062204600F0AF
:100D1000A9FC03E0206A016B2846884770BD70B5C6
:100D200005466C6AA06A40F04000A062E06A40F0AC
:100D30000400E062204600F097FC70BD70B50446E8
:100D4000656A284600F08FFC70BD000038B5044687
:100D50000025002000902068806800F0010078BB2A
:100D60002068806840F001002168886019480068A8
:100D70001949B0FBF1F0009002E00098401E00908D
:100D800000980028F9D101F099FA054619E001F020
:100D900095FA401B022814D92068806800F00100F1
:100DA00078B9A06A40F01000A062E06A40F001004B
:100DB000E06200BF002084F8240000BF012038BD9D
:100DC00005E02068806800F001000028DFD00020E6
:100DD000F5E700008801002040420F002DE9FF5F89
:100DE0000446F74850F82400F64951F82410884288
:100DF0007DD0F548005D002879D1F448807800283E
:100E0000FAD1F34951F82400FFF700FC85B22946D6
:100E1000204603F007FD0120EB4908550020ED496D
:100E200041F82400E64850F82400EB4951F824101A
:100E3000884208DDE34850F82400E14941F82400E5
:100E40000F2006F0C9FA44F62060E44941F8240076
:100E5000E348E44941F8240040F2DC50E24941F81B
:100E60002400D74850F82400D64941F82400002037
:100E7000DE4941F82400DE490855D14850F82400E5
:100E8000DC4951F82410401ADB4941F82400084697
:100E900050F8240000287DD0084650F8240000288F
:100EA00002DD0120D5490855D34850F82400002818
:100EB00002DA0020D1490855CF4951F82400002812
:100EC00001DB014600E04142CD4A42F82410C94806
:100ED00050F82400CB4941F824000121204603F0BA
:100EE00052FAC54850F82400C10F204600E0CCE17A
:100EF00003F00CFAB94830F8240081B2204603F020
:100F00005AFA322006F068FABB4951F8240000284A
:100F100001DB014600E041424908B34A42F824108F
:100F2000114651F82400FFF753FB0546B64850F828
:100F300024102846FFF708FC07D2B34951F82400D3
:100F4000FFF764FBA84941F824000121204603F083
:100F500059FA0121204603F011FA6BE1A64951F834
:100F60002400002801DB014600E041429E4A52F87D
:100F70002420891A9D4A52F8242091427ED3A34905
:100F800031F81400FFF724FB0546964850F824106A
:100F9000284600E06DE1FFF7D7FB70D29C4951F87D
:100FA00024004FF08041FFF7EBF982468F4951F85A
:100FB00024104800FFF70CFB83465146FFF7AEF9BB
:100FC0008146FFF76FFB074607F0ACF80546FFF7D1
:100FD00095FB844941F824008C4931F81400FFF74F
:100FE000F7FA05467F4850F824102846FFF7A2FB81
:100FF00007D2864931F81400FFF7EAFA794941F837
:101000002400784A52F82410724A52F82400FFF75C
:1010100091FB05D2734850F824006E4941F8240032
:101020007C4A52F824106F4A52F82400FFF78CFBD8
:1010300005D2784850F824006A4941F82400764ADD
:1010400052F82410674A52F82400FFF773FB05D2C8
:10105000714850F82400634941F82400614850F871
:1010600024106E48FFF78CF90546FFF7CFFA5B496D
:1010700041F82400084630F8240001E005E08CE047
:1010800081B2204603F097F987E05B4951F82400CC
:10109000002801DB014600E04142534A52F8242077
:1010A000891A524A52F82420914275D8584951F869
:1010B00024004FF08041FFF763F94C49039051F849
:1010C0002400FFF785FA01904B4850F82490B9F1BD
:1010D000000F01DB494601E0C9F100010846FFF7B6
:1010E0006EFA00900199FFF713F94FF080410290DA
:1010F000FFF714F983460399FFF710F98246FFF7CB
:10110000D1FA074607F00EF80546FFF7F7FA35491A
:1011100041F824000A4652F824102E4A52F82400BE
:10112000FFF708FB05D22F4850F82400294941F861
:101130002400384A52F824102A4A52F82400FFF7B3
:1011400003FB05D2334850F82400264941F8240017
:10115000314A52F82410234A52F82400FFF7EAFAE1
:1011600005D22D4850F824001E4941F824001D489E
:1011700050F824102948FFF703F90546FFF746FA0F
:10118000164941F82400084630F8240081B2204670
:1011900003F011F901E0FFE700BF012006F01CF9A0
:1011A000154850F8240000283ADB164850F824006F
:1011B0000E4951F8241008440E4941F8240039E042
:1011C0005C030020B0030020340000200801002050
:1011D00018000020B40000201C99000860000020C6
:1011E0000000FA439800002044000020080300207B
:1011F000070000207803002094030020D000002086
:10120000EC020020CC03002038990008E8030020FD
:101210007C0000205499000870990008002474494B
:101220001C4850F824001C4951F82410401A1B494E
:1012300041F824001A48005D00283FF48FAE194899
:1012400050F8240000280ADB124850F82400124904
:1012500051F824100844114941F8240009E00D48D0
:1012600050F824000C4951F82410401A0B4941F859
:10127000240000200C4941F824000C490855084975
:101280000855052006F0A8F802E00F2006F0A4F8A3
:10129000BDE8FF9FCC030020080300207803002056
:1012A0000700002094030020980000203400002054
:1012B00010B51349098889B2114A126801EB12412D
:1012C0000F4A526801EB12410D4A928892B21144C2
:1012D0000B4A926801EB1241094A128992B21144F9
:1012E000074AD26801EB1241054A928992B28818E6
:1012F000FFF76EF904464FF08241FFF741F810BD49
:10130000BC0C002000BFFEE710B5024800F074FBE3
:1013100010BD00006004002030B590F8405001245A
:10132000AC40C56B6C60046863604468102C04D1E9
:101330000468A2600468E16003E00468A1600468D6
:10134000E26030BD704710B5012000F003FE10BD13
:1013500008490968012282409143064A1160054903
:1013600014310968012282401143024A143211608B
:1013700070470000000401400849096801228240CA
:101380001143064A11600549143909680122824057
:101390001143024A143A11607047000014040140DE
:1013A00072B600BFFEE7000001460020022904D10A
:1013B000034A926802F0010000E000BF00BF7047DE
:1013C0000010014010B504460B46022C08D11BB199
:1013D0000020FFF7D1FF02E00020FFF7B9FF00E097
:1013E00000BF00BF10BD0000F8B504460026002075
:1013F000009000BF94F82400012801D10220F8BD1C
:10140000012084F8240000BF2046FFF731FC064687
:101410002046FFF79BFC0646002E69D1A06A20F407
:10142000885040F00200A062022001F04FF83449D9
:101430000968B1FBF0F04000009002E00098401E07
:10144000009000980028F9D12068806840F00800DA
:101450002168886000F032FF054616E000F02EFF9C
:10146000401B0A2811D92068806800F0080060B18C
:10147000A06A20F0020040F01000A06200BF00202F
:1014800084F8240000BF0120B9E72068806800F0DC
:1014900008000028E2D12068806840F0040021683C
:1014A000886000F00BFF054616E000F007FF401BC8
:1014B0000A2811D92068806800F0040060B1A06A91
:1014C00020F0020040F01000A06200BF002084F86D
:1014D000240000BF012092E72068806800F004002B
:1014E0000028E2D1A06A20F0020040F00100A062D2
:1014F00000BF002084F8240000BF30467FE70000D2
:101500008801002038B5024600230020009000BF6B
:1015100092F82400012801D1022038BD012082F870
:10152000240000BF4868072812D21068406B0C796D
:10153000641E04EB84051F24AC40A0430D796D1E8E
:1015400005EB85050C68AC4020431468606327E018
:1015500048680D2812D21068006B0C79E41F04EB68
:1015600084051F24AC40A0430D79ED1F05EB8505D4
:101570000C68AC4020431468206311E01068C06A16
:101580000C790D3C04EB84051F24AC40A0430D797D
:101590000D3D05EB85050C68AC4020431468E06206
:1015A00008680A2812D31068C0680C780A3C04EB5B
:1015B00044050724AC40A0430D780A3D05EB4505E2
:1015C0008C68AC4020431468E0600FE0106800694C
:1015D0000C7804EB44050724AC40A0430D7805EBE0
:1015E00045058C68AC4020431468206108681028C9
:1015F00002D00868112827D1174C1068A0421ED1CC
:101600001068806800F40000F0B91068806840F449
:1016100000001468A0600868102815D10F48006801
:101620000F4CB0FBF4F000EB80004000009002E0B3
:101630000098401E009000980028F9D104E0906ABC
:1016400040F020009062012300BF002082F82400B7
:1016500000BF184661E70000002401408801002017
:1016600040420F0070477047704700002DE9F0417D
:101670000446002700250026A84614B90120BDE82D
:10168000F081A06810B1207D00B100BFA06A30B920
:101690000020E06284F82400204600F097F82046FD
:1016A000FFF7E6FA0746A06A00F01000002873D1A1
:1016B000002F7ED1A06A20F4885040F00200A06282
:1016C0003F4AD4E90001904208D1E069B0F5402FCB
:1016D00002D14FF4002002E0E06900E0E06901433C
:1016E000207B41EA40000643A068B0F5807F02D02D
:1016F000A068012802D14FF4807000E0002005436B
:10170000207D012811D1207B38B9A069401E4FF4FB
:10171000006141EA4030054307E0A06A40F0200044
:10172000A062E06A40F00100E0622068406820F4B6
:101730006940284321684860206880682149084042
:10174000304321688860A068B0F5807F02D0A0682F
:10175000012802D14FF4807000E00020B0F5807FB6
:1017600003D1208A401E4FEA00582068C06A20F446
:10177000700040EA08002168C86220688068124949
:101780000840B04209D10020E062A06A20F00200C7
:1017900040F00100A06211E00BE0A06A20F002001E
:1017A00040F01000A062E06A40F00100E062012712
:1017B00004E0A06A40F01000A062012738465EE70E
:1017C000003C0140FDF7E1FFFE0E1FFF10B586B0A3
:1017D000044600200290039004900590214920685F
:1017E00088423DD100BF2048806940F400701E4906
:1017F00088610846806900F40070019000BF00BF56
:1018000000BF0846806940F008008861084680698A
:1018100000F00800019000BF00BF03200290039079
:1018200002A9124800F0A4FB1148124908600020E8
:10183000486000210F4881608021C160490001613A
:1018400089004161202181610021C16100F0A0FA7D
:1018500008B1FFF7A5FD00BF06482062446200BF43
:1018600006B010BD0024014000100240000C0140F1
:1018700008000240600400202DE9F04104460D46B6
:101880001646002757492068884203D056492068E9
:10189000884205D15348001D006800F4702000E024
:1018A000002000287ED100BF94F82400012802D136
:1018B0000220BDE8F081012084F8240000BF20460A
:1018C000FFF744FA0746002F6DD1A06A40F6016188
:1018D000884340F48070A06243492068884209D15F
:1018E0004048001D006800F4702008B9012002E0A3
:1018F000002000E0012078B1A06A20F48010A062EE
:101900002068406800F4806000B3A06A20F40050B2
:1019100040F48050A06219E0A06A40F48010A062F8
:1019200030492068884203D02F492068884205D179
:101930002C48001D006800F4806000E0002028B101
:10194000A06A20F4005040F48050A062A06A00F425
:10195000805020B1E06A20F00600E06201E0002043
:10196000E06200BF002084F8240000BF1F48216A05
:1019700088621F48216AC8621E48216A08636FF0A6
:101980000200216808602068806840F48070216847
:101990008860226802F14C0133462A46206A00F032
:1019A0003DFA01E01AE014E02068806800F460204D
:1019B000B0F5602F06D12068806840F4A00021684F
:1019C00088600CE02068806840F48010216888609E
:1019D00005E000BF002084F8240000E0012738461D
:1019E00067E700000024014000280140CD0C0008FA
:1019F0003D0D00081F0D000870B50446E06B05683A
:101A00002068066894F84010042088402840002888
:101A100075D006F004000028FAD02068006800F0B5
:101A2000200028B92068006820F0040021680860C0
:101A3000D5492068884254D9D349783920688842EA
:101A400001D1042049E0D04964392068884201D19D
:101A5000402042E0CC4950392068884201D100152D
:101A60003BE0C9493C392068884202D14FF48040AC
:101A700033E0C54928392068884202D14FF48020DC
:101A80002BE0C14914392068884202D14FF480000C
:101A900023E0BD492068884201D1C0041DE0BB4954
:101AA0002068884201D1042017E0B8491431206829
:101AB000884201D1402010E0B44928312068884292
:101AC00001D1001509E0B1493C312068884202D1BA
:101AD0004FF4804001E04FF48020AC49091F0860BA
:101AE00054E0A94978392068884201D104204AE0AD
:101AF000A54964392068884202D1402043E04CE087
:101B0000A14950392068884201D100153BE09E4927
:101B10003C392068884202D14FF4804033E09A4932
:101B200028392068884202D14FF480202BE0964962
:101B300014392068884202D14FF4800023E0924992
:101B40002068884201D1C0041DE090492068884285
:101B500001D1042017E08D4914312068884201D159
:101B6000402010E0894928312068884201D10015C1
:101B700009E086493C312068884202D14FF4804018
:101B800001E04FF48020804980394860E06A0028F5
:101B900002D02046E16A8847F4E094F84010022021
:101BA00088402840002871D006F002000028FAD0B2
:101BB0002068006800F0200040B92068006820F02C
:101BC0000A0021680860012084F821006E4920681D
:101BD000884254D96C4978392068884201D1022062
:101BE00049E0694964392068884201D1202042E0F7
:101BF000654950392068884201D140153BE062496F
:101C00003C392068884202D14FF4005033E05E49ED
:101C100028392068884202D14FF400302BE05A491D
:101C200014392068884202D14FF4001023E056494D
:101C30002068884201D180041DE054492068884210
:101C400001D1022017E0514914312068884201D1A6
:101C5000202010E04D4928312068884201D14015EC
:101C600009E04A493C312068884202D14FF40050D3
:101C700001E04FF400304549091F086054E0424933
:101C800078392068884202D102204AE057E03E4974
:101C900064392068884201D1202042E03A49503915
:101CA0002068884201D140153BE037493C39206823
:101CB000884202D14FF4005033E03349283920687C
:101CC000884202D14FF400302BE02F4914392068AC
:101CD000884202D14FF4001023E02B49206888424B
:101CE00001D180041DE029492068884201D10220E9
:101CF00017E0264914312068884201D1202010E0E5
:101D0000224928312068884201D1401509E01F4945
:101D10003C312068884202D14FF4005001E04FF47A
:101D2000003019498039486000BF002084F8200045
:101D300000BFA06A30B32046A16A884722E094F829
:101D40004010082088402840E0B106F00800C8B1E3
:101D50002068006820F00E002168086094F84010A8
:101D600001208840E16B48600120A06384F82100D5
:101D700000BF002084F8200000BF206B10B1204677
:101D8000216B884770BD00008000024008040240BB
:101D90000146002209B9012070471E4B086898428D
:101DA0000BD21D4B0868C01A1423B0FBF3F080005F
:101DB000086419480838C8630AE0164B0868C01A56
:101DC0001423B0FBF3F08000086412480838C8639D
:101DD000022081F821000868026843F6F07082430F
:101DE000D1E901031843CB6818430B6918434B69C9
:101DF00018438B691843CB69184302430868026093
:101E000000208863012081F82100002081F8200053
:101E100000BFC1E708040240080002402DE9F0417C
:101E200004460D4616461F464FF0000800BF94F8C2
:101E30002000012802D10220BDE8F081012084F8B1
:101E4000200000BF94F8210001282CD1022084F842
:101E500021000020A0632068006820F001002168B4
:101E600008603B46324629462046FFF755FAE06AAD
:101E700030B12068006840F00E00216808600BE077
:101E80002068006820F0040021680860206800686D
:101E900040F00A00216808602068006840F00100F6
:101EA0002168086006E000BF002084F8200000BF21
:101EB0004FF002084046BFE710B504461F480088AF
:101EC000401C1E4908801E48006840F002001C4962
:101ED00008601C48807888B11B48806800F00100C9
:101EE00058BB0020FFF734FA0021022002F08AFAE2
:101EF000002016498860164988601EE012488068F4
:101F000000F00100C8B10020FFF722FA4FF4C870BA
:101F100005F062FA0021022002F074FA0B48806892
:101F2000002803DD01200A49886003E04FF0FF30FC
:101F30000749886000200549086010BD1001002095
:101F40001404014008010020001001405C0300203F
:101F50007803002010B5044604480068204020B1F2
:101F6000024804602046FFF7A7FF10BD140401409B
:101F70002DE9F847024600239C467BE14FF001081B
:101F800008FA03F4D1F8008008EA0400A0427DD1E9
:101F9000DFF8F4A2D1F80480A8EB0A09D0453AD0C2
:101FA00014DCB8F1030F50D009DCB8F1000F31D0C8
:101FB000B8F1010F1CD0B8F1020F49D120E0B8F1FF
:101FC000110F18D0B8F1120F42D11EE0B9F5881FD9
:101FD00025D006DCB9F5803F20D0B9F5801F37D178
:101FE0001AE0B9F5001F18D0B9F5041F30D117E079
:101FF000D1F80CC02DE0D1F80C8008F1040C28E0D9
:10200000D1F80C8008F1080C23E0D1F80C8008F11D
:102010000C0C1EE000BF00BF00BF00BF00BF00BF30
:10202000D1F80880B8F1000F02D14FF0040C0BE09A
:10203000D1F80880B8F1010F03D14FF0080C1461FA
:1020400002E04FF0080C546103E04FF0000C00E098
:1020500000BF00BFFF2801D8904601E002F104084C
:102060004646FF2802D84FEA830803E0A3F1080898
:102070004FEA88084746D6F800804FF00F0909FA62
:1020800007F928EA09080CFA07F900E07AE048EABB
:102090000908C6F80080D1F8048008F08058B8F12B
:1020A000805F6FD100BFDFF8E481D8F8188048F076
:1020B0000108DFF8D891C9F81880C846D8F8188008
:1020C00008F00108CDF8008000BF00BF4FEAB93822
:1020D0004FEA930958F829504FEA83784FEA187964
:1020E0004FF00F0808FA09F825EA0805DFF8A08183
:1020F000424502D14FF0000824E0DFF898814245C4
:1021000002D14FF001081DE0DFF88C81424502D179
:102110004FF0020816E0DFF88481424502D14FF00B
:1021200003080FE0DFF87881424502D14FF0040840
:1021300008E0DFF87081424502D14FF0050801E068
:102140004FF006084FEA83794FEA197908FA09F83F
:1021500048EA0505DFF850814FEA930948F829500D
:10216000D1F8048008F48018B8F5801F0BD1DFF88F
:102170003C81D8F8008048EA0008DFF83091C9F8BF
:1021800000800AE075E0DFF82481D8F8008028EAB2
:102190000008DFF81891C9F80080D1F8048008F42D
:1021A0000018B8F5001F0ED1DFF8008108F104080F
:1021B000D8F8008048EA0008DFF8F09009F1040937
:1021C000C9F800800DE0DFF8E48008F10408D8F8D1
:1021D000008028EA0008DFF8D49009F10409C9F862
:1021E0000080D1F8048008F40038B8F5003F0ED123
:1021F000DFF8B880A8F10408D8F8008048EA0008A1
:10220000DFF8A890A9F10409C9F800800DE0DFF813
:102210009C80A8F10408D8F8008028EA0008DFF8BC
:102220008C90A9F10409C9F80080D1F8048008F461
:102230008038B8F5803F0ED1DFF87080A8F108082B
:10224000D8F8008048EA0008DFF86090A9F1080992
:10225000C9F800800DE0DFF85480A8F10808D8F82C
:10226000008028EA0008DFF84490A9F10809C9F8BD
:1022700000805B1CD1F8008028FA03F8B8F1000F49
:102280007FF47CAEBDE8F88700001110001002401A
:1022900000080140000C0140001001400014014002
:1022A00000180140001C01400800014008040140E2
:1022B0000AB1016101E00B04036170470148006845
:1022C000704700007C01002003480068034909783A
:1022D00008440149086070477C0100208401002007
:1022E00010B50848006840F0100006490860032057
:1022F00000F0D8F80F2000F007F800F055F80020A3
:1023000010BD000000200240F0B587B00446002652
:102310000027002500BF1F48806940F400601D4968
:1023200088610846806900F40060009000BF00BF2B
:1023300001A902A800F0B4FA00F0EAFA064616482D
:10234000B6FBF0F0471E15481549086040F2E7312A
:102350001348C1604760002101618160816100F024
:10236000DBFD054695B90E4800F05CFE05466DB9EB
:10237000192000F049F8102C07D20022214619201C
:1023800000F052F80748046000E00125284607B035
:10239000F0BD00000010024040420F00002C014040
:1023A000440D00208001002008B500BF144880695A
:1023B00040F00100124988610846806900F0010080
:1023C000009000BF00BF00BF0846C06940F08050C9
:1023D000C8610846C06900F08050009000BF00BF8F
:1023E00000220F21901E00F01FF800BF0549486829
:1023F00020F0E06040F00070486000BF08BD0000C1
:10240000001002400000014001460846002809DB98
:1024100000F01F0301229A4043099B0003F1E023CF
:10242000C3F8002100BF70472DE9F05F80460D46DC
:102430001646002703F0E6FA074639462A46334691
:1024400001F00700C0F1070ABAF1040F02D94FF0FA
:10245000040A01E0C0F1070AD14600F1040ABAF10A
:10246000070F02D24FF0000A01E0A0F1030AD446A0
:102470004FF0010A0AFA09FAAAF1010A0AEA020A65
:102480000AFA0CFA4FF0010B0BFA0CFBABF1010B43
:102490000BEA030B4AEA0B042146404603F0BAFA62
:1024A000BDE8F09F00BF00F00702064B19684FF629
:1024B000FF031940044B0B4343EA0221014B19600F
:1024C00000BF70470CED00E00000FA052DE9F04771
:1024D00006464FF00008002500270024A146042EE0
:1024E00037D004DC012E3CD0022E6CD160E0082EE7
:1024F00033D0102E67D136484468006800F08070F1
:1025000008B33448C4F38341475C04F4803078B1A5
:102510002F484068C0F340402F4911F8008004F470
:10252000803040B12D48B0FBF8F000FB07F502E029
:102530002B4807FB00F52648406800F48000B0F502
:10254000800F01D1A94603E068000321B0FBF1F937
:102550003AE000F0EDF9814636E000F0E9F9814615
:1025600032E01B48046A04F44070B0F5807F05D166
:1025700004F0020010B14FF4004918E004F4407078
:10258000B0F5007F07D11248406A00F0020010B198
:1025900049F640490BE004F44070B0F5407F06D1A5
:1025A0000B48006800F4003008B14FF224490BE0FA
:1025B00000F0AEF906494968C1F38131491C490070
:1025C000B0FBF1F900E000BF00BF4846BDE8F0876E
:1025D00000100240EA990008FA99000800127A00F7
:1025E00000093D00F8B5044600260025207800F0DB
:1025F000010000286BD000274348C06900F08050DC
:1026000070B900BF4048C06940F080503E49C86181
:102610000846C06900F08050009000BF00BF01274D
:102620003A48006800F48070B0B93848006840F457
:10263000807036490860FFF741FE064606E0FFF766
:102640003DFE801B642801D90320F8BD2F48006897
:1026500000F480700028F2D02B48006A00F4407526
:102660002DB3A08800F44070A84220D02648006A0C
:1026700020F44075012026490860002008602248A7
:10268000056205F0010090B1FFF718FE064608E06C
:10269000FFF714FE801B41F28831884201D90320E4
:1026A000D3E71948006A00F002000028F0D016486D
:1026B000006A20F440706168084313490862012FE2
:1026C00004D10846C06920F08050C86100BF20785E
:1026D00000F00200022807D10B48406820F4404077
:1026E000A168084308494860207800F010001028CD
:1026F00007D10548406820F4800061690843024919
:1027000048600020A1E70000001002400070004077
:102710004004424270B504460D460CB9012070BD1C
:102720005A48006800F00700A8420ED257480068D7
:1027300020F007002843554908600846006800F06B
:102740000700A84201D00120E9E7207800F002004C
:1027500002281DD1207800F00400042805D14C483F
:10276000406840F4E0604A494860207800F0080082
:10277000082805D14648406840F460504449486004
:102780004348406820F0F000A16808434049486091
:10279000207800F0010078B36068012806D13C4839
:1027A000006800F4003090B90120B8E760680228A2
:1027B00006D13748006800F0007040B90120AEE74C
:1027C0003348006800F0020008B90120A7E730484C
:1027D000406820F00300616808432D494860FFF716
:1027E0006DFD064609E0FFF769FD801B41F2883167
:1027F000884202D9032092E707E02548406800F0AC
:102800000C006168B0EB810FEDD12048006800F04A
:102810000700A8420ED91D48006820F00700284391
:102820001A4908600846006800F00700A84201D075
:10283000012074E7207800F00400042807D1144830
:10284000406820F4E060E16808431149486020785E
:1028500000F00800082808D10D48406820F46050B6
:10286000216940EAC1000A49486000F061F808495E
:102870004968C1F30311074A515CC8400649086022
:1028800006480068FFF740FD002048E700200240AE
:1028900000100240FC9900088801002080010020FF
:1028A0000F2202600D4A526802F0030242600B4A96
:1028B000526802F0F0028260084A526802F4E06254
:1028C000C260064A526802F46052D2080261044AA9
:1028D000126802F007020A60704700000010024010
:1028E0000020024001480068704700008801002075
:1028F00000B5FFF7F7FF04494968C1F30221034A15
:10290000515CC84000BD0000001002400C9A000855
:1029100000B5FFF7E7FF04494968C1F3C221034A44
:10292000515CC84000BD0000001002400C9A000835
:1029300070B500210022002400230020134D696897
:1029400001F00C05F5B1042D02D0082D19D101E0DC
:102950000F4819E00F4DC1F38346AB5D01F480359C
:1029600055B10A4D6D68C5F340450B4E725D084D7B
:102970005D43B5FBF2F402E0084D03FB05F420468D
:1029800002E000BF024800BF00BF70BD001002405F
:1029900000127A00D8990008E899000800093D0063
:1029A000F8B504460CB90120F8BD207800F001000C
:1029B000002878D0F848406800F00C0004280CD0BB
:1029C000F548406800F00C00082811D1F248406832
:1029D00000F48030B0F5803F0AD1EF48006800F481
:1029E000003000285FD0606800285CD10120DBE760
:1029F00000BF6068B0F5803F06D1E748006840F44A
:102A00008030E549086028E0606858B9E24800680D
:102A100020F48030E04908600846006820F48020F7
:102A200008601AE06068B0F5A02F0BD1DA480068A2
:102A300040F48020D84908600846006840F480309F
:102A400008600AE0D448006820F48030D249086069
:102A50000846006820F48020086000BF606888B1E4
:102A6000FFF72CFC054606E0FFF728FC401B642816
:102A700001D9032098E7C848006800F40030002816
:102A8000F2D010E0FFF71AFC054606E0FFF716FC4F
:102A9000401B642801D9032086E7BF48006800F482
:102AA00000300028F2D1207800F00200022857D12F
:102AB000B948406800F00C0050B1B748406800F0D9
:102AC0000C00082818D1B448406800F4803098B948
:102AD000B148006800F0020020B12069012801D04F
:102AE000012061E7AC48006820F0F800616940EA25
:102AF000C100A949086033E02069E8B10120A74975
:102B00000860FFF7DBFB054606E0FFF7D7FB401B3D
:102B1000022801D9032047E79F48006800F002001F
:102B20000028F2D09C48006820F0F800616940EA73
:102B3000C1009949086013E0002098490860FFF738
:102B4000BDFB054606E0FFF7B9FB401B022801D993
:102B5000032029E79048006800F002000028F2D125
:102B6000207800F0080008282DD1A069B8B1012014
:102B70008B490860FFF7A2FB054606E0FFF79EFBC6
:102B8000401B022801D903200EE78348406A00F069
:102B900002000028F2D0012001F04EFC13E00020DA
:102BA0007F490860FFF78AFB054606E0FFF786FBD2
:102BB000401B022801D90320F6E67748406A00F05E
:102BC00002000028F2D1207800F00400042873D11C
:102BD00000277148C06900F0805070B900BF6E488E
:102BE000C06940F080506C49C8610846C06900F077
:102BF0008050009000BF00BF01276A48006800F4C1
:102C00008070B0B96748006840F48070654908601A
:102C1000FFF754FB054606E0FFF750FB401B642816
:102C200001D90320C0E65F48006800F480700028E6
:102C3000F2D000BFE068012806D15748006A40F092
:102C400001005549086227E0E06858B95248006A17
:102C500020F00100504908620846006A20F0040094
:102C6000086219E0E06805280BD14B48006A40F083
:102C70000400494908620846006A40F00100086201
:102C80000AE04548006A20F001004349086208460E
:102C9000006A20F00400086200BFE068A0B1FFF7FE
:102CA0000DFB054609E0FFF709FB401B41F28831A7
:102CB000884202D9032077E622E03748006A00F014
:102CC00002000028EFD012E0FFF7F8FA054608E00E
:102CD000FFF7F4FA401B41F28831884201D9032002
:102CE00062E62D48006A00F002000028F0D1012FB2
:102CF00005D12948C06920F080502749C86100BF2C
:102D0000E069C8B32448406800F00C00082860D08F
:102D1000E069022848D1002020490866FFF7CEFA72
:102D2000054606E0FFF7CAFA401B022801D9032036
:102D30003AE61948006800F000700028F2D1206AD5
:102D4000B0F5803F07D11448406820F40030A168F6
:102D5000084311494860D4E9080108430E4949680D
:102D600021F4741108430C49486001200B4908669E
:102D7000FFF7A4FA054607E03DE0FFF79FFA401B86
:102D8000022801D903200FE60348006800F0007014
:102D90000028F2D02FE00000001002400000424264
:102DA0008004424200700040002014490866FFF78A
:102DB00085FA054606E0FFF781FA401B022801D993
:102DC0000320F1E50E48006800F000700028F2D101
:102DD00011E0E069012800D1E6E50948466806F4FB
:102DE0008031206A814204D106F47011606A814208
:102DF00001D00120D8E50020D6E5000000004242C5
:102E0000001002407047704710B50346002200BF13
:102E100093F83C00012801D1022010BD012083F865
:102E20003C0000BF22F0FF00CC6840EA040222F41C
:102E300040708C6840EA040222F480604C6840EAEA
:102E4000040222F400600C6840EA040222F480507C
:102E50000C6940EA040222F400504C6940EA040282
:102E600022F48040CC6940EA04021868426400BF42
:102E7000002083F83C0000BF00BFCEE730B502461B
:102E80000B4600BF92F83C00012801D1022030BD62
:102E9000012082F83C0000BF022082F83D0010684B
:102EA00044681068816824F070041868044310684E
:102EB0004460144D1068A84213D0134D1068A84206
:102EC0000FD01068B0F1804F0BD0104D1068A842A1
:102ED00007D00F4D1068A84203D00E4D1068A842CD
:102EE00005D121F0800158680143106881600120FC
:102EF00082F83D0000BF002082F83C0000BF00BF08
:102F0000C5E70000002C01400034014000040040EF
:102F100000080040000C004010B504460CB9012028
:102F200010BD94F83D0028B9002084F83C002046EC
:102F300000F026F8022084F83D00211D206802F0F0
:102F4000A5F9012084F8460000BF84F83E00012165
:102F50003F200155402001554120015500BF00BFD1
:102F6000012084F8420043200155442001554520AA
:102F7000015500BF012084F83D000020D0E700008B
:102F800038B504462068B0F1804F16D100BF224802
:102F9000C06940F001002049C8610846C06900F0DE
:102FA0000100009000BF00BF002205211C20FFF798
:102FB0003BFA1C20FFF728FA2CE0184920688842C9
:102FC00016D100BF1448C06940F002001249C86120
:102FD0000846C06900F00200009000BF00BF002258
:102FE00005211D20FFF720FA1D20FFF70DFA11E043
:102FF0000B49206888420DD100BF0748806940F422
:103000000050054988610846806900F4005000902E
:1030100000BF00BF38BD00000010024000040040A7
:1030200000340140014691F83D00012801D0012003
:103030007047022081F83D000868C06840F0010038
:103040000B68D860164B0868984213D0154B086877
:1030500098420FD00868B0F1804F0BD0124B08682F
:10306000984207D0114B0868984203D0104B08686B
:1030700098420CD10868806800F00702062A0CD03C
:103080000868006840F001000B68186005E00868F7
:10309000006840F001000B6818600020C8E70000DD
:1030A000002C0140003401400004004000080040B2
:1030B000000C00402DE9F04104460D46002700BFFA
:1030C00094F83C00012802D10220BDE8F0810120E3
:1030D00084F83C0000BF022084F83D002068866828
:1030E00026F0770626F47F462068866028685028F8
:1030F00033D00CDC202850D004DC00284BD0102822
:1031000051D149E0302849D040284CD139E06028DD
:103110002DD0702807D0B0F5805F03D0B0F5005FE8
:1031200041D10DE041E0D5E902136A68206802F060
:1031300014F92068866846F077062068866034E0D7
:10314000D5E902136A68206802F007F920688068F0
:1031500040F480402168886027E0EA686968206858
:1031600002F0ECF95021206802F002F91DE0EA6853
:103170006968206802F0F5F96021206802F0F8F82B
:1031800013E0EA686968206802F0D8F940212068F5
:1031900002F0EEF809E000BF00BF00BF2968206818
:1031A00002F0E6F801E0012700BF00BF012084F82B
:1031B0003D0000BF002084F83C0000BF384684E793
:1031C000704770B504462068C5682068066906F037
:1031D0000200022819D105F00200022815D1401F73
:1031E00021680861012020772068806900F00300D1
:1031F00018B12046FFF7E4FF05E0204600F01CF977
:10320000204600F0F1F90020207706F004000428A1
:1032100019D105F00400042815D1C04321680861C4
:10322000022020772068806900F4407018B12046A1
:10323000FFF7C6FF05E0204600F0FEF8204600F04C
:10324000D3F90020207706F00800082819D105F0EE
:103250000800082815D1C0432168086104202077A0
:103260002068C06900F0030018B12046FFF7A8FFEE
:1032700005E0204600F0E0F8204600F0B5F9002017
:10328000207706F01000102819D105F01000102842
:1032900015D1C04321680861082020772068C069E3
:1032A00000F4407018B12046FFF78AFF05E0204681
:1032B00000F0C2F8204600F097F90020207706F0D1
:1032C000010048B105F0010030B16FF00100216844
:1032D0000861204600F004FA06F08000802809D139
:1032E00005F08000802805D1C04321680861204690
:1032F000FFF788FD06F04000402809D105F04000A6
:10330000402805D1C04321680861204600F0F4F947
:1033100006F02000202809D105F02000202805D142
:10332000C043216808612046FFF76DFD70BD0000B5
:1033300010B586B0044600200290039004900590DA
:103340002068B0F1804F16D100BF3548806940F049
:103350000400334988610846806900F00400019048
:1033600000BF00BF022002900390059002A92D48E3
:10337000FEF7FEFD52E02C492068884217D100BFBD
:103380002748806940F00400254988610846806923
:1033900000F00400019000BF00BF40200290022016
:1033A0000390059002A91F48FEF7E2FD36E01F4991
:1033B0002068884217D100BF1948806940F0040096
:1033C000174988610846806900F00400019000BF39
:1033D00000BF0420029002200390059002A911482A
:1033E000FEF7C6FD1AE012492068884216D100BFD8
:1033F0000B48806940F010000949886108468069DF
:1034000000F01000019000BF00BF40200290022099
:103410000390059002A90748FEF7AAFD06B010BD6B
:10342000001002400008014000040040000C004071
:10343000003401400010014070472DE9F04104467E
:103440000D461646002700BF94F83C00012802D123
:103450000220BDE8F081012084F83C0000BF36B1B5
:10346000042E1BD0082E31D00C2E5ED145E029460B
:10347000206801F087FF2068806940F0080021681B
:1034800088612068806920F00400216888612068D4
:103490008069296908432168886148E029462068D5
:1034A00001F0A8FF2068806940F40060216888610D
:1034B0002068806920F480602168886120688069C4
:1034C000296940EA01202168886130E029462068A6
:1034D00001F0CEFF2068C06940F008002168C86193
:1034E0002068C06920F004002168C8612068C069B4
:1034F000296908432168C86119E02946206801F05C
:10350000F3FF2068C06940F400602168C86120684A
:10351000C06920F480602168C8612068C069296999
:1035200040EA01202168C86101E0012700BF00BF17
:1035300000BF002084F83C0000BF384689E710B582
:1035400004460CB9012010BD94F83D0028B90020B4
:1035500084F83C00204600F025F8022084F83D0065
:10356000211D206801F092FE012084F8460000BF72
:1035700084F83E0001213F200155402001554120A3
:10358000015500BF00BF012084F8420043200155CF
:10359000442001554520015500BF012084F83D001D
:1035A0000020D0E738B504460D492068884215D17F
:1035B00000BF0C48C06940F008000A49C8610846CD
:1035C000C06900F00800009000BF00BF0022052184
:1035D0003220FEF729FF3220FEF716FF38BD00002B
:1035E000000C0040001002407047000070B5044617
:1035F0000D4615B994F83E000BE0042D02D13F2092
:10360000005D06E0082D02D14020005D01E0412070
:10361000005D012801D0012070BD1DB9022084F891
:103620003E000EE0042D03D102213F20015508E0A9
:10363000082D03D102214020015502E00221412042
:10364000015501222946206801F076FE1F492068B5
:10365000884203D01E492068884201D1012000E041
:10366000002028B12068406C40F400402168486484
:1036700016492068884213D01549206888420FD027
:103680002068B0F1804F0BD012492068884207D0E3
:1036900011492068884203D01049206888420CD123
:1036A0002068806800F00706062E0CD020680068AD
:1036B00040F001002168086005E02068006840F0E3
:1036C0000100216808600020A6E70000002C0140EE
:1036D000003401400004004000080040000C00409D
:1036E00010B5044603492068884201D1FEF7ECFD7D
:1036F00010BD0000002C0140704710B504460CB905
:10370000012010BDA06900B100E000BF94F84100A5
:1037100028B9002084F84000204600F029F8242031
:1037200084F841002068C06820F400502168C86017
:10373000204601F061FF2068006920F49040216874
:1037400008612068406920F02A00216848612068EB
:10375000C06840F400502168C860002060642020E8
:1037600084F8410084F842000020606300BFC8E78D
:1037700010B586B004460020029003900490059096
:103780003949206888422FD100BF3848806940F409
:103790008040364988610846806900F48040019085
:1037A00000BF00BF00BF0846806940F00400886188
:1037B0000846806900F00400019000BF00BF481572
:1037C0000290022003900320059002A92848FEF7EA
:1037D000CFFB4FF48060029000200390049002A978
:1037E0002348FEF7C5FB3DE022492068884239D1D5
:1037F00000BF1E48C06940F480201C49C8610846CB
:10380000C06900F48020019000BF00BF00BF0846DF
:10381000806940F0100088610846806900F010005F
:10382000019000BF00BF0815029002200390032002
:10383000059002A91048FEF79BFB4FF40060029030
:1038400000200390049002A90B48FEF791FB00BFF3
:103850000A49486820F0300040F0E06040F0100075
:10386000486000BF06B010BD0038014000100240A3
:1038700000080140004800400010014000000140E5
:103880002DE9F84F04460E46174699464FF0000AB8
:1038900094F84100202850D106B117B90120BDE8A5
:1038A000F88F00206064212084F84100FEF706FDB7
:1038B0008246A784E784A068B0F5805F04D12069C0
:1038C00010B90025B04602E035464FF000081EE072
:1038D0005346002280212046CDF8009001F00AFFD7
:1038E00020B1202084F841000320D8E745B9B8F87A
:1038F0000000C0F308002168486008F1020803E0F6
:103900002878216848606D1CE08C401EE084E08CC3
:103910000028DDD15346002240212046CDF80090FA
:1039200001F0E8FE20B1202084F841000320B6E732
:10393000202084F841000020B1E70220AFE700BF5B
:10394000FEE700002DE9FC474448454988604548AA
:103950004549886000BFC82003F03EFD42488068AA
:10396000424989688842F6D1642003F035FDFDF7AD
:103970009FFC3F490860084600683E4908603E4990
:1039800008603E48006838498860002450E0FDF730
:103990008FFC37490860082C2EDA3448816804EB24
:1039A000C40000EB0410364A02EB0020A0F25230B3
:1039B000814221DD2D48816804EBC40000EB041036
:1039C00002EB002000F25230814210DA28480168F0
:1039D00029480068FCF79CFC05462A49FCF7B4FE20
:1039E0000AD2012028490855601CC4B204E0002016
:1039F00025490855601CC4B21D480068FCF752FEFA
:103A000005460E4619498868FCF7D9FD82461F49CC
:103A1000FCF7B6FC8146FCF745FE07463A460B46E6
:103A20001BA0CDE9005601F0BBFF0A2003F0D4FC37
:103A30000D4880680D4989688842A8D100BFC82018
:103A400003F0CAFC08488068084989688842F6D1B2
:103A5000124803498860BDE8FC87000000401C460E
:103A60001800002080F3FFFF5C0300207803002093
:103A7000240100203C010020500100204C010020C6
:103A8000C0F9FFFF0000FA43540100200000C842C3
:103A90002532662C2533660A0000000000409C4653
:103AA00010B50948006800F4807058B14FF4C87030
:103AB00002F091FC0448001D006840F0807002494B
:103AC000091D086010BD00000C0801400348006893
:103AD00040F4807001490860704700001008014000
:103AE00038B50446084A0021084803F0CBFC0849D1
:103AF000086000204FF4E13301222146009002F0DB
:103B000051FF02F0ABFC38BD149C000815410008C1
:103B1000E00200200EB5002000900190029057486E
:103B200057490860811556488160012101730021C1
:103B300001754FF46021C161002051494860102196
:103B40004F480161FDF792FD08B1FDF729FC0820FF
:103B50000090012001900720029069464848FDF737
:103B6000D1FC08B1FDF71CFC0220019069464448D5
:103B7000FDF7C8FC08B1FDF713FC0320019069466E
:103B80003F48FDF7BFFC08B1FDF70AFC0420019097
:103B900069463B48FDF7B6FC08B1FDF701FC05207E
:103BA000019069463648FDF7ADFC08B1FDF7F8FB1A
:103BB0000620019069463248FDF7A4FC08B1FDF7E4
:103BC000EFFB0720019069462D48FDF79BFC08B1EB
:103BD000FDF7E6FB0820019069462948FDF792FCB5
:103BE00008B1FDF7DDFB09200090019069462448EB
:103BF000FDF788FC08B1FDF7D3FB0A200190694668
:103C00001F48FDF77FFC08B1FDF7CAFB0B200190B0
:103C100069461B48FDF776FC08B1FDF7C1FB0C2097
:103C2000019069461648FDF76DFC08B1FDF7B8FB39
:103C30000D20019069461248FDF764FC08B1FDF7BC
:103C4000AFFB0E20019069460D48FDF75BFC08B103
:103C5000FDF7A6FB0F20019069460948FDF752FCCD
:103C600008B1FDF79DFB1020019069460448FDF75F
:103C700049FC08B1FDF794FB0EBD00000024014093
:103C80003004002008B500BF0A48406940F0010038
:103C9000084948610846406900F00100009000BFF3
:103CA00000BF002205210B20FEF7BEFB0B20FEF714
:103CB000ABFB08BD0010024000B585B000200190AC
:103CC00002900390049000BF4348806940F02000B8
:103CD000414988610846806900F02000009000BFDB
:103CE00000BF00BF0846806940F0100088610846A8
:103CF000806900F01000009000BF00BF00BF0846C0
:103D0000806940F0040088610846806900F0040082
:103D1000009000BF00BF00BF0846806940F0080067
:103D200088610846806900F00800009000BF00BF6D
:103D3000002240F2A9112948FEF7BAFA00223021E8
:103D40002748FEF7B5FA00224FF4E0512548FEF768
:103D5000AFFA01200190244802900020039001A9AD
:103D60001F48FEF705F906200190002002900390FD
:103D700001A91B48FEF7FCF840F2A91001900120B0
:103D80000290002003900220049001A91348FEF73E
:103D9000EFF83020019001200290002003900220D3
:103DA000049001A90E48FEF7E3F84FF4E0500190AB
:103DB00001200290002003900220049001A90948EC
:103DC000FEF7D6F8002205210620FEF72DFB06207F
:103DD000FEF71AFB05B000BD0010024000080140CC
:103DE00000100140000C01400000211000B58DB012
:103DF000002009900A900B900C90079008901C21CD
:103E00006846FCF728FA4FF08040214908604820B6
:103E1000486000211E48816040F2E731C160002106
:103E2000016180218161FFF777F808B1FDF7B8FAE9
:103E30004FF48050099009A91548FFF73BF908B1E4
:103E4000FDF7AEFA1248FFF77AFB08B1FDF7A8FAC2
:103E5000202007900020089007A90D48FFF70EF8D2
:103E600008B1FDF79DFA6020009040F2F310019038
:103E7000002002900490042269460548FFF7DDFA0D
:103E800008B1FDF78DFA0248FFF752FA0DB000BDF8
:103E9000A404002000B58DB0002009900A900B907A
:103EA0000C90079008901C216846FCF7D4F9224832
:103EB000224908604820486000212048816040F283
:103EC000E731C1600021016180218161FFF724F8A1
:103ED00008B1FDF765FA4FF48050099009A9174819
:103EE000FFF7E8F808B1FDF75BFA1448FFF727FB86
:103EF00008B1FDF755FA202007900020089007A987
:103F00000E48FEF7BBFF08B1FDF74AFA60200090AB
:103F100040F2F310019000200290049000226946C4
:103F20000648FFF78AFA08B1FDF73AFA0348FFF7A7
:103F3000FFF90DB000BD000000040040EC040020BB
:103F400000B589B00020079008901C216846FCF756
:103F500082F91A481A490860482048600021184828
:103F6000816040F2E731C1600021016180218161FF
:103F7000FFF7E5FA08B1FDF713FA202007900020BB
:103F8000089007A90E48FEF779FF08B1FDF708FA77
:103F90006020009040F2F310019000200290049005
:103FA000082269460648FFF748FA08B1FDF7F8F914
:103FB0000348FFF7BDF909B000BD0000000C004048
:103FC0003405002000B595B0002011901290139098
:103FD00014900F9010901C2108A8FCF73CF92021A8
:103FE0006846FCF738F92C482C490860482048609E
:103FF00000212A48816040F2E731C160002101615F
:10400000416180218161FEF787FF08B1FDF7C8F9A2
:104010004FF48050119011A92048FFF74BF808B1D8
:10402000FDF7BEF91D48FFF78AFA08B1FDF7B8F9A8
:1040300020200F90002010900FA91848FEF71EFFB7
:1040400008B1FDF7ADF960200890002009900A90B2
:104050000B900C900D900E90002208A90F48FFF7CE
:10406000ECF908B1FDF79CF9002000900190029056
:10407000039004904FF4005005900020079069468B
:104080000648FEF7C1FE08B1FDF78AF90348FFF7BD
:104090004FF915B000BD0000003401407C05002040
:1040A00010B50B480B4908604FF4E130486000211F
:1040B00008488160C16001610C214161002181617A
:1040C000C161FFF71AFB08B1FDF76AF910BD0000E6
:1040D00000380140C405002010B50B480B490860AA
:1040E0004FF4E1304860002108488160C1600161FF
:1040F0000821416100218161C161FFF7FEFA08B129
:10410000FDF74EF910BD0000004800400C060020ED
:1041100000BFFEE700BF02F0B5FC0A2003F05CF927
:10412000F9E700001CB51421002000F07BFB4FF4E0
:104130007A71012000F076FB44F62061022000F045
:1041400071FB1448182100234FF48072CDE9001050
:1041500011A1144805F0FCF8134908600D48001D32
:10416000182101231A02CDE9001010A10D4805F015
:10417000EFF8114908600748083018210223DA01D6
:10418000CDE900100DA1074805F0E2F80E490860DE
:104190001CBD0000140400205461736B4E616D65FA
:1041A00031000000CD630008140100205461736BDE
:1041B0004E616D6532000000180100205461736B80
:1041C0004E616D65330000001C010020044600BFF5
:1041D00024B1012C03D0022C09D104E000BF2046F9
:1041E00000F03EF904E02046FCF7F8FD00E000BFD7
:1041F000EEE7000010B5044600203B490855FDF7E6
:10420000A7F80021204600F0FDF8012037490855A5
:1042100000212046FDF7D6F80121204600F0AEF837
:104220000121204600F072F80A2003F0D5F80021A1
:10423000204600F0A8F8C821204600F0BCF820462F
:10424000FDF7B2F8C8B90021204600F05FF80A2057
:1042500003F0C2F80121204600F0D4F84FF41670A4
:1042600003F0BAF80021204600F0CCF801212046E6
:1042700000F04CF8962003F0AFF801212046FDF73E
:10428000A1F80121204600F0BDF80020184941F8AE
:1042900024000120174941F8240006E000201649B7
:1042A00041F82400142003F097F8124850F8240035
:1042B0000028F3D1104941F82400104941F82400A6
:1042C0000B4941F824000E4941F824000D490855D6
:1042D0000120054908550020054941F824000A49F4
:1042E00008550249085510BD0101002008010020B1
:1042F0005C0300207803002008030020EC0200206B
:10430000B0030020D0000020FA00002020B10128D6
:1043100011D002282DD11DE031B1174A126842F4A4
:104320000022154B1A6005E0134A126842F0080299
:10433000114B1A601EE031B10F4A126842F40012AC
:104340000D4B1A6005E00C4A126842F020020A4B3D
:104350001A600FE031B1084A126842F00102064BC0
:104360001A6005E0044A126842F48032024B1A6077
:1043700000E000BF00BF70471008014000B900E036
:1043800000BF00BF704770B505460C4625B1012D32
:1043900006D0022D08D108E0204600F019FF08E001
:1043A000204600F09FFE04E000BF204600F024FEFF
:1043B00000BF00BF70BD70B505460C4625B1012D8C
:1043C0000BD0022D1BD111E0264604EBD670C0F3B2
:1043D0004F01204600F0F4FE12E0264604EBD670B2
:1043E000C0F34F01204600F075FE09E0264604EBBD
:1043F000D670C0F34F01204600F0F9FD00E000BF89
:1044000000BF70BD70B505460C4625B1012D06D024
:10441000022D0CD107E0204600F0B0FE08E0204657
:1044200000F036FE04E0204600F0C4FD00E000BFCE
:1044300000BF70BD00BFFEE708B508490968C9089C
:104440004FF47A72B1FBF2F14143009100BF00BF1B
:1044500000994A1E00920029F9D108BD8801002068
:104460002DE9FE4F0446DB4850F82400002872D0A6
:10447000D948005D00286ED1D84951F82400FCF7D6
:10448000C5F885B22946204600F0CCF90120D24972
:1044900008550020D24941F824004FF4FA60D14970
:1044A00041F82400D048D14941F824006420D04983
:1044B00041F824000020CF4941F82400CE49085596
:1044C000C44850F82400CD4941F824000121204679
:1044D000FFF759FFCA48015D2046FFF717FFC9489B
:1044E00050F82410C848FBF74BFF0646FCF78EF83F
:1044F00085B229462046FFF75EFF322002F06CFFAE
:1045000001212046FFF73AFFBC4850F8240040083C
:10451000B74941F8240051F82400FCF759F8054642
:10452000BA4850F824102846FCF70EF907D2B749CC
:1045300051F82400FCF76AF8AD4941F82400012144
:104540002046FFF75FFF25E1B148005D20B1002064
:10455000AF49085523E138E1A64850F82400A449A2
:1045600051F8241088426FD2A24951F82410480013
:10457000FCF72EF88246A74850F824105046FBF767
:10458000CDFE8146FCF78EF8074603F0CBFD0546CD
:10459000FCF7B4F8954941F824000A4652F8241073
:1045A0008F4A52F82400FCF7C5F805D28F4850F81E
:1045B00024008B4941F82400974A52F824108B4A72
:1045C00052F82400FCF7C0F805D2934850F82400B4
:1045D000864941F824008B4A52F82410834A52F845
:1045E0002400FCF7A7F805D2864850F824007F493C
:1045F00041F82400894931F81400FBF7E9FF05462A
:104600007A4850F824102846FCF794F807D28349DA
:1046100031F81400FBF7DCFF744941F824007348BB
:1046200050F824107848FBF7ABFE0546FBF7EEFF89
:104630006C4941F82400084630F8240081B2204635
:10464000FFF7B9FEA3E0FFE76C4850F82400684983
:1046500051F82410401A674951F82410884239D380
:104660006E4931F81400FBF7B3FF06463146664841
:10467000FBF786FE0546FBF7C9FF5A4941F82400BF
:10468000084630F8240081B22046FFF794FE06E089
:104690000020584941F82400052002F09DFE4D48B5
:1046A00050F824004FF6FF718842F1D0494850F885
:1046B000240000286BD14E4850F8240040004F4998
:1046C00041F824004A4850F82400401C494941F868
:1046D00024005CE04F4951F824004FF08041FBF783
:1046E0004FFE4449029051F82400FBF771FF434903
:1046F000019051F82400FBF76BFF00900199FBF744
:1047000007FE83464FF08041FBF708FE8246029980
:10471000FBF704FE8146FBF7C5FF074603F002FDE9
:104720000546FBF7EBFF314941F824003A4A52F8BD
:1047300024102E4A52F82400FCF706F805D2364819
:1047400050F82400294941F824002E4A52F8241038
:10475000264A52F82400FBF7EDFF05D2294850F80D
:104760002400224941F82400204850F8241026480B
:10477000FBF706FE0546FBF749FF1A4941F82400FE
:10478000084630F8240081B22046FFF714FE0520C9
:1047900002F022FE1848005D00283FF4D5AE00BFAD
:1047A0000F2002F019FE00200A4941F824001C489D
:1047B000015D2046FFF7E2FD0020074908550E493C
:1047C00008550F2002F008FE02E00F2002F004FE60
:1047D000BDE8FE8F5C03002034000020180000209C
:1047E000B4000020600000200000C04098000020BD
:1047F000440000200803002007000020EC020020F5
:10480000DE000020709900080050C3473899000866
:10481000D70000207C00002054990008E803002005
:10482000E50000202DE9F04104460D460E4830F821
:104830001400A84215D00D4850F824104FF08040C5
:10484000FBF76CFD064605FB05F0FBF7B8FE0746D7
:104850003146FBF795FD064941F82400024820F84F
:104860001450BDE8F0810000E803002038990008EA
:104870007C0000202DE9F04F8BB04FF00009FE487E
:10488000007828B9002003F0A7FE0BB0BDE8F08F38
:104890000124D4E240F2DC5002F09EFDF648005DB7
:1048A00000287DD0F548005D0028FAD04FF4C850AC
:1048B0006043F349886000BFC82002F08DFDF048D6
:1048C0008068F04989688842F6D140F2DC5002F0F5
:1048D00083FD2246ECA1F04801F072F8EF48016830
:1048E000EF480068FBF71AFD0546FBF776FEE44942
:1048F00048600020EB490870EB48008800F0FEFAA1
:1049000000BFC82002F068FDDD484068DD49496805
:104910008842F6D1002000F0F1FA40F2DC5002F0BB
:104920005BFD0020D649886000BFC82002F054FD1E
:10493000D3488068D34989688842F6D14FF47A70A9
:1049400002F04AFDD948DA490860DA480168D748D8
:10495000FBF716FD0546FBF740FEC949086000BF9E
:10496000C82002F039FDC6480068C6490968884277
:10497000F6D1D148CE4908604FF47A7002F02CFD90
:104980004FF4C8506043BE49886000BFC82002F0A1
:1049900023FDBB488068BB4989688842F6D100E0A6
:1049A00044E240F2DC5002F017FD0020C3490880C9
:1049B000C34908602246C3A1B74801F001F8FCF7DB
:1049C00077FCC449086008460068C3490860C348CA
:1049D000AB490860B448008800F090FA00BFFCF7CB
:1049E00067FCBC49086008460168BB480068FBF7E3
:1049F000C7FC0790FBF756FECDE9080102F046FC24
:104A000007460022B64BFBF7F9FC0546FBF731FEE3
:104A10001FFA80FB5846FBF7DBFD8246A349FBF7F4
:104A2000AFFCB0490860B0490868FBF7D1FD824689
:104A3000A04801685046FBF771FC80469B49FBF794
:104A40006DFC0746FBF7E2FD0646FBF7C1FD054698
:104A50009649FBF795FC9A490860A2480068A3496B
:104A6000964A128841F8220095480068A049934A66
:104A7000128841F8220097480068FBF713FE0546AC
:104A80000E4698480068FBF70DFE07463A460B466F
:104A900098A0CDE9005600F083FF9949914800683D
:104AA000FBF752FE77D209F10109B9F1050F73DB6B
:104AB0009348944908600020714908609249087041
:104AC000642000F01BFA4FF47A7002F085FC7B48FA
:104AD000008800B28D4908804FE08C480088401E55
:104AE00000B28A49088087480068FBF7DBFD05466D
:104AF0000E467E49854AB2F9002051F822008449C9
:104B0000FBF706FC8246FBF7CDFD21F0004107468E
:104B10002A463346FBF7DAFD17D274497B4AB2F9CD
:104B2000002051F822007A49FBF7F2FB0746FBF719
:104B3000B9FD21F000410546FBF7E0FD7149086031
:104B40007248B0F900007349088068496F4AB2F9A9
:104B5000002051F822006E49FBF7ECFD0DD26448AD
:104B60006A49B1F9001050F821006B4941F824005E
:104B70004FF0FF306549088004E06448B0F9000058
:104B80000028AADC00BF61480088002804D1C720A3
:104B90005E49088051E0F0E0DBE05A480068FBF72E
:104BA00081FD05460E465149584AB2F9002051F898
:104BB00022005749FBF7ACFB8246FBF773FD21F05F
:104BC000004107462A463346FBF780FD17D2474986
:104BD0004E4AB2F9002051F822004D49FBF798FBEC
:104BE0000746FBF75FFD21F000410546FBF786FD18
:104BF000444908604548B0F90000464908803B49EF
:104C0000424AB2F9002051F822004149FBF792FDD7
:104C10000DD237483D49B1F9001050F821003E4906
:104C200041F824004FF0FF30384908800CE0374845
:104C30000088401E00B2354908803448B0F90000B1
:104C40001E4909888842A8DC00BF3048B0F900003E
:104C50001A49098888427CD12A480068FBF722FD5E
:104C6000074688462149294AB2F9002051F8220016
:104C70002749FBF74DFB51E0540100205C01002067
:104C80005C030020780300202564BAC5B1ADDDCDFA
:104C9000C8A12F3000000000540600202801002089
:104CA00030010020380100203A01002000007A4441
:104CB000180000202C0100200000A0414401002029
:104CC000340100202564BAC5B1ADD6D0BACD2F309D
:104CD00000000000240100203C010020F0F16300EE
:104CE00000408F4040010020080300207C06002087
:104CF0009C090020252E33662C2533660A0000000F
:104D00009A99993E74010020390100207001002019
:104D1000713D8A3E78010020040D00208246FBF799
:104D2000C1FC21F0004105463A464346FBF7CEFC64
:104D300019D25349534AB2F9002051F8220052497E
:104D4000FBF7E6FA0746FBF7ADFC21F0004105460C
:104D500000E014E0FBF7D2FC4C4908604948B0F988
:104D600000004B4908804B484949B1F9001050F800
:104D70002100494941F8240001E04FF0000947486B
:104D80000088401C80B245490880C82801DB00200B
:104D90000880322002F020FB414800684149096840
:104DA00088427FF41CAE404951F824000021FBF7F3
:104DB000C1FC35D03C4951F82400FBF773FC824616
:104DC0008B46354951F8240038490968FBF7A0FAA9
:104DD0000190FBF767FC0546354A364BFBF70EFBA7
:104DE0000746354A354BFBF709FB52465B46CDE992
:104DF0000201FBF775FB0022314BCDE90401FBF703
:104E0000FDFACDE90601FBF715FC0890FBF7D7FB8F
:104E10002C490990FBF7B4FA2B4941F824000CE027
:104E20001D4850F824002149086006E027A12948C0
:104E300000F0C6FD00201A490860601CC4B2082CAE
:104E4000FFF628AD002000F059F840F2DC5002F0E7
:104E5000C3FA00201249886000BFC82002F0BCFAE3
:104E60000F4880680F4989688842F6D14FF47A70FC
:104E700002F0B2FA002003F0AFFB00BF05E500002E
:104E80007C06002070010020713D8A3E74010020E4
:104E9000780100209C090020040D0020440100201E
:104EA0005C03002078030020E40C00206401002053
:104EB0007B14AE47E17A943FCDCCCCCCCC0C4C40AB
:104EC00000408F4000247449240D0020BFD5CEBB84
:104ED0002F3000005406002010B504460548FCF7AA
:104EE00083FA102204490348FCF7C6FC00F09CFC3E
:104EF00010BD000030040020BC0C002001490968EE
:104F0000486370477C05002010B54FF0E020006931
:104F100004F0AEFA012801D003F0F8FE10BD00B590
:104F200095B028210BA8FBF796F9142106A8FBF7EA
:104F300092F918216846FBF78EF901200B900004C6
:104F40000C9000200D9001200F9002201290C103C0
:104F500013914FF4E01114910BA8FDF721FD08B156
:104F6000FCF71EFA0F200690022007900020089000
:104F70004FF48060099000200A90022106A8FDF7F6
:104F8000C9FB08B1FCF70CFA0220009080030290E4
:104F90006846FDF727FB08B1FCF702FA15B000BD23
:104FA0007047000010B50248FEF70BF910BD000075
:104FB000440D002068B14FF08041098841F00101A3
:104FC0004FF0804211801146098C41F0100111848C
:104FD0000CE04FF08041098C21F010014FF080422D
:104FE00011841146098821F00101118070474FF0AA
:104FF000804290851187704768B14FF08041898960
:1050000041F004014FF0804291811146098A21F05C
:10501000050111820CE04FF08041898921F00401E3
:105020004FF0804291811146098A21F005011182D9
:105030007047000010B51248FEF7C3F84FF08040EB
:10504000006920F005004FF0804108610D4880683C
:105050000D498968884205D20A488068401C094980
:1050600088600CE00020FFF7A5FF01200749887049
:105070008007006920F005004FF08041086110BDF5
:10508000A404002008030020EC02002007000020F8
:1050900070B10F49098841F001010D4A11800C4996
:1050A0002031098841F00101094A203211800DE0C8
:1050B00007492031098821F00101054A2032118079
:1050C0000349098821F00101014A1180704700005D
:1050D00000040040024A1080014A083211807047E3
:1050E0002C04004060B10D49098841F002010B4ACF
:1050F0001180111D098821F00301121D11800BE0A0
:105100000649098821F00201044A1180111D09880D
:1051100021F00301121D1180704700000C040040B3
:1051200010B51148FEF74DF81048006820F0030054
:105130000E4908600E4840680E494968884205D209
:105140000B484068401C0A4948600BE00020FFF70C
:105150009FFF0120084948700448006820F00300C0
:105160000249086010BD0000EC040020100400405B
:1051700008030020EC0200200700002070B10F4956
:10518000098841F001010D4A11800C49203109883C
:1051900041F48071094A203211800DE00749203125
:1051A000098821F48071054A203211800349098859
:1051B00021F00101014A118070470000000C0040FD
:1051C000024A1080014A1032118070472C0C0040B6
:1051D00060B10D49098841F008010B4A1180111D89
:1051E000098821F00901121D11800BE00649098888
:1051F00021F00801044A1180111D098821F00901DC
:10520000121D1180704700000C0C004010B51148B1
:10521000FDF7D7FF1048006820F009000E4908602C
:105220000E4800680E490968884205D20B4800689C
:10523000401C0A4908600BE00020FFF79FFF012097
:10524000084908700448006820F009000249086015
:1052500010BD000034050020100C004008030020A1
:10526000EC0200200700002010B50748008800F07D
:10527000010038B10448008820F00100024908808C
:1052800002F080FE10BD00001014004010B502684E
:10529000244B98420ED0244B98420BD0B0F1804F53
:1052A00008D0224B984205D0214B984202D0214B86
:1052B000984203D122F070024B681A43194B98426E
:1052C0000ED0194B98420BD0B0F1804F08D0174B3D
:1052D000984205D0164B984202D0164B984203D103
:1052E00022F44072CB681A4322F080034C6943EAEF
:1052F000040202608B68C3620B688362094B9842A8
:1053000002D0094B984201D10B6903630123436129
:10531000036903F001031BB1036923F00103036177
:1053200010BD0000002C014000340140000400408A
:1053300000080040000C004030B501F01F050124BA
:1053400004FA05F3046A9C430462046A01F01F0531
:1053500002FA05F52C43046230BD30B50C46816875
:1053600021F47F4142EA032525432943816030BD72
:105370000A46816821F0700142F0070319438160F9
:105380007047000030B5026A056A25F00105056224
:105390004368846924F0700424F003040D682C43EE
:1053A00022F002028D682A43104DA84200D103E08A
:1053B0000F4DA84206D100BF22F00802CD682A4353
:1053C00022F00402094DA84202D0094DA84207D19B
:1053D00023F4807323F400734D692B438D692B43B1
:1053E000436084614D684563026230BD002C01401A
:1053F0000034014030B5026A056A25F010050562E7
:105400004368846924F4E04424F440740D6844EA59
:10541000052422F020028D6842EA0512124DA842AE
:1054200000D103E0114DA84207D100BF22F0800255
:10543000CD6842EA051222F040020B4DA84202D08C
:105440000A4DA84209D123F4806323F400634D6917
:1054500043EA85038D6943EA8503436084614D68AF
:105460008563026230BD0000002C01400034014021
:1054700030B5026A056A25F4807505624368C4691F
:1054800024F0700424F003040D682C4322F400720D
:105490008D6842EA0522124DA84200D103E0114D69
:1054A000A84207D100BF22F40062CD6842EA05227B
:1054B00022F480620A4DA84202D00A4DA84209D1C6
:1054C00023F4805323F400534D6943EA05138D6997
:1054D00043EA05134360C4614D68C563026230BD91
:1054E000002C01400034014030B5036A056A25F400
:1054F000805505624468C26922F4E04222F4407299
:105500000D6842EA052223F400538D6843EA05330F
:10551000084DA84202D0084DA84204D124F480448A
:105520004D6944EA85144460C2614D6805640362B4
:1055300030BD0000002C01400034014030B50B4666
:105540001446026A056A25F001050562816921F0A9
:10555000F00141EA041122F00A021A438161026259
:1055600030BD30B50B461446026A056A25F01005B9
:105570000562816921F4704141EA043122F0A00200
:1055800042EA03128161026230BD00BF00BF0268BF
:105590000C3252E8002F22F4907102680C3242E87B
:1055A0000013002BF3D100BF00BF00BF026814320C
:1055B00052E8002F22F001010268143242E8001381
:1055C000002BF3D100BF016B01290ED100BF00BF3A
:1055D00002680C3252E8002F22F0100102680C32EF
:1055E00042E80013002BF3D100BF202180F84210C5
:1055F000002101637047000070B504462168096905
:1056000021F44051E2681143226811612269A168C6
:105610001143626941EA02052168C96841F20C62DE
:10562000914329432268D1602168496921F440717E
:10563000A2691143226851612D4A2168914202D129
:10564000FDF766F901E0FDF753F900EBC00101EB4E
:10565000001162689200B1FBF2F100EBC00202EBB4
:10566000001263689B00B2FBF3F26423B2FBF3F217
:1056700002EBC20303EB0212A1EB8201322202EB26
:1056800001116422B1FBF2F101F0F00100EBC00264
:1056900002EB001263689B00B2FBF3F26423B2FBDF
:1056A000F3F201EB021200EBC00101EB00116368A1
:1056B0009B00B1FBF3F100EBC00303EB0013666842
:1056C000B600B3FBF6F36426B3FBF6F303EBC306B5
:1056D00006EB0313A1EB8301322303EB01116423D7
:1056E000B1FBF3F101F00F0111442268916070BD2C
:1056F000003801402DE9F84304460D461746984608
:10570000089E31E0701C70B3FCF7D8FDA0EB0800D8
:10571000B04200D816B90320BDE8F8832068C068FD
:1057200000F00400F8B1802D1ED0402D1CD0206860
:105730000068C0F3C000B0B100BF00200090206836
:105740000068009020684068009000BF00BF2046BD
:10575000FFF71BFF0820606400BF002084F84000B2
:1057600000BF0120D8E7FFE7206800682840A84272
:1057700001D1012000E00020B842C3D00020CBE7D7
:1057800010B52548008800F0010048B12248008883
:10579000C0B2224908802048001D0088C0B208809D
:1057A0001E48008838B100201C4908801C48006849
:1057B000401C1B49086018480C30008800F020008D
:1057C00030B11548008800F0200008B102F0E2FB7B
:1057D00011480C30008800F0800030B10E4800887D
:1057E00000F0800008B102F0DDFB0B480C300088AF
:1057F00000F0400020B90848008800F0400048B19F
:1058000005480C30008820F0400003490C31088026
:10581000FEF746F910BD000000380140DC02002010
:10582000D802002000BFFEE744A1474800F0C8F8B6
:105830000120FEF755F94548454908604548464965
:105840000860FEF76FFC00204449086048608860EB
:105850000220FEF7CFFCFEF775F841484149086089
:10586000414808604148C860FBF722FD4049086094
:10587000084600683F49086000BF3F48007800289C
:1058800040D000203C4908703449886000BFC820DF
:1058900001F0A2FD31488068384989688842F6D114
:1058A0002B4801684FF07E50FAF738FD0446FAF7AE
:1058B00094FE2A49486000203149087000BFC82082
:1058C00001F08AFD254840682C4949688842F6D194
:1058D000254824490860204801682348FAF750FD0C
:1058E0000446FAF77AFE1D49086000BFC82001F09F
:1058F00073FD1A480068214909688842F6D11848A2
:10590000184908601F48007850B11F4A00211F48FD
:1059100001F0B8FD1E49086000201A49087009E02E
:105920001C48807830B11CA1074800F049F80220DB
:10593000FEF760FCC82001F04FFD9EE7BDF8C8EB04
:10594000CFB5CDB32F300000540600200086A1470C
:105950002801002096093F3C2C0100205C03002018
:105960000000A0411800002000007A4400409C453F
:10597000240100203C0100207A010020780300204F
:105980003801002068010020B4990008754800081B
:105990006C010020FA000020D5D2C1E32F300000B6
:1059A0000FB4054B10B503A9044A029800F086F91C
:1059B00010BC5DF814FB0000156F0008E402002025
:1059C0000FB4084B10B504A902AA039800F076F9A9
:1059D000044602A9002000F0F4FC204610BC5DF84B
:1059E00014FB0000C3630008002809DB00F01F025D
:1059F000012191404209920002F1E022C2F8001117
:105A00007047000002480068C0F3022070470000A1
:105A10000CED00E010B5002804DB0A07130E054A60
:105A2000135406E00A07140E034A00F00F031B1F6D
:105A3000D45410BD00E400E018ED00E0EFF3058061
:105A400070472DE9F0414F1E00EBC7010446D1E934
:105A5000000115461E4637F006020DD02A46334691
:105A6000FAF7CCFC7F1E04EBC703D3E90023FAF757
:105A700050FF37F00602F1D1022F25D0042F13D0AA
:105A8000062F18BFBDE8F0812A463346FAF7B6FC68
:105A9000D4E90A23FAF73DFF2A463346FAF7AEFC6B
:105AA000D4E90823FAF735FF2A463346FAF7A6FC6D
:105AB000D4E90623FAF72DFF2A463346FAF79EFC6F
:105AC000D4E90423FAF725FF2A463346FAF796FC71
:105AD000D4E90223FAF71DFF2A463346FAF78EFC73
:105AE000D4E90023BDE8F041FAF713BF00221346C2
:105AF00010460149FAF7F4BC0000F03F0122FAF722
:105B0000AFBF0022134610461146FAF7E9BC02E087
:105B100008C8121F08C1002AFAD170477047002038
:105B200001E001C1121F002AFBD170470149086042
:105B300070470000E80200202DE9FF5F82B00021DD
:105B4000DDE90430020DDDF840B0034318D044F61F
:105B50001050A2F2FF3242431514119801281FD0B1
:105B6000A5EB0B00401C5FEA000A4FF000064E4F09
:105B7000DFF83891B046504615D5CAF1000413E05D
:105B8000119801244AA3012801D16FEA0B01029860
:105B9000119AC0E90031C0E9024206B0BDE8F09FA9
:105BA000CBF10000DFE704460021404A491842EBF0
:105BB0000450CDE9001012E0E00707D032463B4622
:105BC00040464946FAF71AFC8046894632463B462B
:105BD00010461946FAF712FC06460F466410002CD0
:105BE000EAD1DDE90401DDE90023BAF1000F06DAAC
:105BF000FAF704FC42464B46FAF700FC05E0FAF7D8
:105C00006FFC42464B46FAF76BFC04460E460022F8
:105C1000284BFAF7B7FF03D84FF0FF30014607E0F3
:105C20000022254B20463146FAF773FEFAF791FF22
:105C3000102409E0002C0ADB0A220023FAF7A4FD55
:105C4000039B30321A55641E50EA0102F2D1641CE3
:105C5000039AC4F111031444119A012A03D00122BA
:105C600008430DD10AE0084304D000204FF0110B87
:105C7000119072E7A3EB0B056D1E0DE05B4504DD93
:105C80004FF0000205F1010504E003DA4FF00002D5
:105C9000A5F10105002AECD002981199C0E9023162
:105CA000C0E9004579E70000000014400000F03F23
:105CB000300000000000F0430000E03F2DE9FF4FFE
:105CC00095B09A46884606460025EEE1252877D10C
:105CD00000242746F94A0121039400E0044316F802
:105CE000013F203B01FA03F01042F7D130782A2817
:105CF00011D06FF02F033078A0F13002092A16D8A6
:105D0000039A44F0020402EB820203EB42021044C5
:105D1000761C0390EFE758F8042B0392002A03DA6D
:105D2000504244F40054039044F00204761C30784E
:105D30002E2816D116F8010F44F004042A280DD09D
:105D40006FF02F023078A0F13003092B09D807EB50
:105D5000870302EB4303C718761CF3E758F8047B6C
:105D6000761C30786C280FD006DC4C2817D06828B9
:105D70000DD06A2814D104E0742810D07A280FD1ED
:105D80000DE044F400140AE044F4801401E044F40B
:105D900040147278824202D104F58014761C761C7D
:105DA000307866280BD013DC582877D009DC00281F
:105DB00075D04528F6D04628F4D047281AD193E16B
:105DC00018E0632835D0642879D0652812D18BE19A
:105DD000702873D008DC6728F1D069286FD06E284E
:105DE0000DD06F2806D1ACE073282CD0752874D064
:105DF000782853D05246179990476D1C54E1C4F34C
:105E00000250022809D003280DD0D8F80010042829
:105E10000DD00D6008F1040846E1D8F80010EA172B
:105E2000C1E90052F6E7D8F800100D80F2E70D70D6
:105E3000F0E718F8041B8DF8001000208DF8010021
:105E4000EB46012003E058F804BB4FF0FF30610738
:105E50004FF0000102D40DE009F101018946B94279
:105E60000FDA8145F8DB1BF809100029F4D108E0AE
:105E700009F1010189468142FADB1BF8091000296A
:105E8000F6D103985346A0EB090721463846179AE6
:105E900000F080FA284400EB090507E044E008E13F
:105EA0000DE01BF8010B524617999047B9F1010913
:105EB000F7D2534621463846179AF2E039E00A21D4
:105EC000C4F302524FF0000B0091022A06D058F89A
:105ED000040BC117032A09D00AE023E008F10700E8
:105EE00020F00702F2E80201904605E000B2C11777
:105EF000042A01D140B2C117002906DA0A4600215E
:105F0000404261EB02012D2202E0220504D52B2242
:105F10008DF80420012203E0E20701D02022F7E7F8
:105F2000914657E00A2100E010214FF0000B00914C
:105F30000BE010214FF0000B44F0040408270091FF
:105F400003E008204FF0000B0090C4F30252022A35
:105F500005D058F8040B0021032A08D008E008F106
:105F6000070020F00702F2E80201904603E080B249
:105F7000042A00D1C0B24FF0000922072AD5327896
:105F8000702A07D0DDF800C08CF0100C5CEA0B0C16
:105F900005D00EE040228DF80420012208E050EAEE
:105FA000010306D030238DF804308DF8052002223D
:105FB0009146009B83F0080353EA0B030AD150EA91
:105FC000010201D1620705D530228DF804204FF07F
:105FD00001097F1E3278582A04D039A20C920CAAEB
:105FE00002920BE03BA2F9E75B46009AFAF7CCFB82
:105FF0000C9B9B5C029A521E0292137050EA0102A3
:10600000F2D1029804A9081A00F1200B600702D50A
:1060100024F4803400E001275F4502DDA7EB0B008C
:1060200000E0002000EB0B01009003984944401A67
:106030000390E00306D453462146179A039800F0D4
:10604000A9F90544002706E001A85246C05D17994A
:1060500090476D1C7F1C4F45F6DBE0030CD5534683
:106060002146179A039800F095F9054404E0302082
:106070005246179990476D1C0099481E00900029C0
:10608000F5DC08E00298029952460078491C02911A
:10609000179990476D1CBBF10001ABF1010BF1DCCE
:1060A0005BE100F065F90544761C307800287FF448
:1060B0000DAE19B02846BDE8F08F00000928010098
:1060C000303132333435363738396162636465666E
:1060D0000000000030313233343536373839414230
:1060E0004344454600000000600700D4062708F13D
:1060F000070020F00700F0E80223804603F0004C80
:106100005FEA0C0001D097A009E0200501D596A018
:1061100005E0E00701D095A001E0AFF24C0013903C
:10612000307823F0004365280CD006DC452809D0E0
:1061300046281DD047287FD13BE0662818D0672825
:106140007AD136E00021112F01DB112000E0781C0C
:10615000CDE9000104A90CA8FFF7EEFCDDE90D0173
:106160000C9A4FF0000B07F10109109200914EE0DC
:106170004FF000400097CDE9011004A90CA8FFF7EB
:10618000DBFCDDE90D020C9B0F994FF0000B9146F3
:106190001093009211B9791C00EB0109B7EB0900CB
:1061A00003D4C0F1FF3B07F10109A9EB07000190FF
:1061B00042E0012F00DA01270021112F01DD11201B
:1061C00000E03846CDE9000104A90CA8FFF7B4FCB3
:1061D000DDE90D010C9A00914FF0000BB9461092C9
:1061E00021070FD4009A4A4503DA914601E0A9F14C
:1061F0000109B9F1010F05DD109AA9F10101515C06
:106200003029F4D0B84202DA10F1040F03DA012188
:10621000CDE9011010E0002803DC8344A9EB000164
:1062200002E0411C494500DD8946A0EB0B00401C03
:1062300001904FF000400290200705D40198484596
:1062400002DB4FF0FF30019000208DF84B000298E8
:106250000DF14B07B0F1004F25D002200C902B2000
:106260000D90029800280CDA404202902D200D90EB
:1062700007E00A210298FAF771FA3031029007F824
:10628000011D0C99481E0C900029F2DC0298002890
:10629000EFD1791E0D980870307800F0200040F0A2
:1062A000450007F8020D11A8C01BC01D02901398ED
:1062B000007800B1012000EB0901019801EBE071C9
:1062C000029801440398401A401E0390E00306D44C
:1062D00053462146179A039800F05CF8054413983A
:1062E000007818B15246179990476D1CE00323D5EA
:1062F00053462146179A039800F04CF805441BE0DA
:10630000BBF1000F07DB0098584504DD1098179982
:1063100010F80B0001E01799302052469047019881
:106320000BF1010B401E05F10105019004D12E2057
:106330005246179990476D1CB9F10001A9F1010966
:10634000DEDC05E017F8010B5246179990476D1CEB
:106350000299481E02900029F4DC53462146179A00
:1063600003989EE62D0000002B0000002000000096
:106370002DE9F041044600251E461746880404D442
:1063800005E039462020B0476D1C641EF9D528462B
:10639000BDE8F0812DE9F041044600251E469046F7
:1063A000C80301D5302700E02027880404D505E084
:1063B00041463846B0476D1C641EF9D52846BDE8F5
:1063C000F0810A68531C0B60107070470446254624
:1063D000E8B2FDF7FBFE3CE000BF00BF00BF00BF1E
:1063E00000BF00BF00BF00BF00BF00BF00BF00BFB5
:1063F00000BF00BF00BF00BF00BF00BF00BF00BFA5
:1064000000BF00BF00BF00BF00BF00BF00BF00BF94
:1064100000BF00BF00BF00BF00BF00BF00BF00BF84
:1064200000BF00BF00BF00BF00BF00BF00BF00BF74
:1064300000BF00BF00BF00BF00BF00BF00BF00BF64
:1064400000BF00BF00BF00BF00BF00BF00BF00BF54
:1064500000BF011EA0F10100BED1704710B500249D
:1064600006480078012806D10548006880470020CA
:106470000249087000E00624204610BD1E020020DC
:10648000240200202DE9F05F06460D464FF0000B78
:106490002888052848D170784FEA0029B07840EA6A
:1064A000090909F101001FFA80F9F0780402307936
:1064B0000443012C35DBB4F5FA6F32DA374600209D
:1064C0002880012007F8010B2888401C288004F050
:1064D000070040B12046E11704EB5171C910491C77
:1064E00001F0FF0805E02046E11704EB5171C1F30C
:1064F000C70807F8018B2888401C28800023224603
:106500004946384600F0FCFB8246BAF1000F04D041
:10651000504601F025FD834608E028884044288045
:1065200004E04FF0030B01E04FF0030B5846BDE8C9
:10653000F09F2DE9F05F06460D464FF0000B2888CE
:10654000052847D170784FEA0029B07840EA090958
:1065500009F101001FFA80F9F07804023079044350
:10656000012C34DBB4F5FA6F31DA3746002028808D
:10657000022007F8010B2888401C288004F007003F
:1065800040B12046E11704EB5171C910491C01F0DC
:10659000FF0805E02046E11704EB5171C1F3C7087D
:1065A00007F8018B2888401C288022464946384637
:1065B00000F0F4FB8246BAF1000F04D0504601F01F
:1065C000CFFC834608E028884044288004E04FF050
:1065D000030B01E04FF0030B5846BDE8F09F2DE997
:1065E000F04705460C464FF0000A2088052837D1B1
:1065F00068784FEA0028A87840EA080808F1010006
:106600001FFA80F8E87806022E79012E25DB7D2E10
:1066100023DC2F4600202080032007F8010B208870
:10662000401C20807006000E07F8010B2088401CDB
:106630002080002332464146384600F0E1FB814687
:10664000B9F1000F04D0484601F08AFC824609E007
:10665000208800EB4600208004E04FF0030A01E0B0
:106660004FF0030A5046BDE8F0872DE9F047054694
:106670000C464FF0000A2088052837D168784FEA89
:106680000028A87840EA080808F101001FFA80F8FD
:10669000E878060228790643012E24DB7D2E22DAD3
:1066A0002F4600202080042007F8010B2088401C82
:1066B00020807006000E07F8010B2088401C208007
:1066C00032464146384600F0F9FB8146B9F1000FE9
:1066D00004D0484601F044FC824609E0208800EBE3
:1066E0004600208004E04FF0030A01E04FF0030A67
:1066F0005046BDE8F0872DE9FC5F04460D460020BA
:10670000009028880A285DDB60784FEA002AA0788C
:1067100040EA0A0A0AF101001FFA80FAE07806024C
:106720002079064360794FEA002BA07940EA0B0BF1
:106730000BF101001FFA80FBE0790702207A074382
:10674000607A0190012E3BDB7D2E39DC012F37DB97
:10675000792F35DC79000198814231D101233A4605
:10676000594604F10A0000F04BFB8146B9F1000FD5
:106770001ED1A04600202880172008F8010B288889
:10678000401C28807006000E08F8010B2888401C69
:106790002880002332465146404600F031FB8146B6
:1067A000B9F1000F04D12888022101FB06002880DE
:1067B000B9F1000F06D0484601F0D2FB009001E08D
:1067C000032000900098BDE8FC9F000070B50546CE
:1067D0000C46064802880649681CF9F723FD034861
:1067E0000088401C2080002070BD00000C020020AA
:1067F000603800202DE9F84304460F464FF00008AA
:106800003888052829D160780502A0780543681CDE
:1068100085B22079F0B9E078FF2801D0E078C8B9D6
:1068200000208DF80100E078FF2803D101208DF8C9
:10683000000002E000208DF8000001231A462946DE
:10684000684600F05DFA06464EB1304601F088FB1E
:10685000804604E04FF0030801E04FF00308404693
:10686000BDE8F8832DE9F04104460F464FF00008DB
:106870003888052812D160780502A0780543681C85
:1068800085B201231A462946E01C00F0B9FA0646F3
:1068900036B1304601F064FB804601E04FF003085A
:1068A0004046BDE8F0812DE9F05F05460E464FF009
:1068B000000B3088052839DD68780702A87807437F
:1068C000781C87B2E87804022879044395F805A07B
:1068D00004F0070040B12046E11704EB5171C910E4
:1068E000491C01F0FF0805E02046E11704EB517157
:1068F000C1F3C708012C16DBB4F5F66F13DCD045E5
:1069000011D1012322463946A81D00F0F9F981462C
:10691000B9F1000F04D0484601F022FB834607E09E
:106920000520308004E04FF0030B01E04FF0030B33
:106930005846BDE8F09F2DE9F04704460E464FF05B
:10694000000A3088062828DB60780702A078074311
:10695000781C87B2E07805022079054394F8059009
:10696000012D17DB782D15DC6806000E484511D186
:1069700001232A463946A01D00F042FA8046B8F1AC
:10698000000F04D0404601F0EBFA824607E00520F4
:10699000308004E04FF0030A01E04FF0030A504654
:1069A000BDE8F0872DE9F04705460C4616461F4620
:1069B000DDF820904FF000081CB1012C01DBF72C12
:1069C00002DD4FF0020835E01C48047005BB1C488E
:1069D0001C4908601C481D4908601D481D49086085
:1069E0001D481E49086000201D4908601D481E49B9
:1069F00008601E481E4908601E481F4908604B4633
:106A00003A4631460D48007800F0D2F8804602E060
:106A10004FF0020800BF00BFB8F1000F0AD101F02B
:106A20004BFF10B94FF0030804E014480570012033
:106A3000134908704046BDE8F08700001C020020A2
:106A4000D56C000824020020F16C00082802002008
:106A5000456C000820020020FD6B00082C0200207D
:106A600030020020558A0008340200201D8B0008E7
:106A700038020020DD8A00083C0200201D020020B0
:106A80001E02002038B500253F48007808B10620D6
:106A900038BD684601F0FEFE002872D09DF8000067
:106AA00030B1012805D0022818D0032868D166E04B
:106AB00066E0364A36493748374B1B6898470546E3
:106AC0005DB93448007835490978884202D03148A8
:106AD000007810B9022001F0F7FE51E02C48006860
:106AE00000782F49087001202E490870002417E013
:106AF0002D4810F8340000B914E02B4810F8340089
:106B00002749097888420AD1274800EBC4001F4969
:106B100042681F48006890472249087002E0641CE0
:106B2000102CE5DB00BF1B48007830B31D4800780F
:106B3000C8B10020154908801948007840F080014C
:106B4000124802880088401C104B188010480068CA
:106B5000815414480178184602880088401C188027
:106B60000B480068815409480288094801680B48AD
:106B700000780E4B1B689847054601E001E000BF16
:106B800000BF002084E700001E020020CE0200208B
:106B9000C8020020CC0200202C0200201C02002091
:106BA000CD020020D0020020480200202002002058
:106BB0002DE9F04781460E4614461F464FF0000867
:106BC0003B4608222146304601F096FE10B94FF0B0
:106BD00003080EE0B4F5964F01D9232503E06000C9
:106BE0000549B1FBF0F5A8B201F00AFF08B94FF072
:106BF00003084046BDE8F087A07F17002DE9F0416B
:106C000004460D46164600270C480088042810DB71
:106C10000A4801880A4801F0ABFA50B908480078E0
:106C2000207006480088C01E30800548401C28603F
:106C300000E005273846BDE8F08100001A02002078
:106C4000803800202DE9F04105460E4617464FF0EA
:106C500000081B48007801282CD1701E19490860D3
:106C60000120194908801748006805700846008807
:106C700038440880084601881248006801F078FA14
:106C8000044611490888411C0F4B19800F490C54C8
:106C9000221219460888411C19800C490A541E20EA
:106CA00000F09AFB01200A4908700121002001F040
:106CB000DDFA01E04FF005084046BDE8F081000034
:106CC0001102002014020020180200208038002049
:106CD0001002002010B50020044908700021012096
:106CE00001F0C4FA01F008FB10BD00001102002001
:106CF00010B50021084601F0B9FA01F0E1FA10BD23
:106D00002DE9F04705460E46174699464FF0000A12
:106D10003CB23220FFF75FFB012E37DBF019512820
:106D200034DC701E1FFA80F8B9F1000F03D0B9F1FE
:106D3000010F2AD116E012E0082C01DD082000E046
:106D40002046C2B24146144801F01EFF05F8010B6F
:106D5000A4F1080004B208F108001FFA80F8002C22
:106D6000EADC12E00EE015F8013B082C01DD0820FA
:106D700000E02046C2B24146074801F01AFFA4F1E4
:106D8000080004B2002CEEDC00BF01E04FF0010A65
:106D90005046BDE8F0870000CA3A00202DE9F047D0
:106DA00005460C4616464FF0000937B23220FFF771
:106DB00012FB012C1CDBA019512819DC601E1FFAE4
:106DC00080F812E0082F01DD082000E03846C2B24A
:106DD00041460A4801F0D8FE05F8010BA7F108006A
:106DE00007B208F108001FFA80F8002FEADC01E082
:106DF0004FF001094846BDE8F0870000C03A002086
:106E00002DE9F04704460F46164698464FF0000914
:106E10003220FFF7E0FA012F34DBB819512831DCBA
:106E2000781E05B2B8F1000F03D0B8F1010F28D1D8
:106E300012E00EE0204830F81500001204F8010BB3
:106E40001D4810F8150004F8010B681C05B2701EEF
:106E500086B2002EEEDC14E011E014F8011B0802EB
:106E6000154921F8150014F8010B31F815100843E5
:106E7000114921F81500681C05B2701E86B2002E5B
:106E8000EBDC16E0B7F57A7F11DDB81940F2D1716D
:106E900088420CDCA7F2E93005B2B8F1000F03D04C
:106EA000B8F1010F02D100E000E000BF01E04FF0B7
:106EB00001094846BDE8F087203A00202DE9F0415D
:106EC00004460D4616464FF000083220FFF783FABD
:106ED000012D17DBA819512814DC681E07B20EE03B
:106EE0000B4830F81700001204F8010B084810F89E
:106EF000170004F8010B781C07B2701E86B2002E32
:106F0000EEDC01E04FF001084046BDE8F0810000F2
:106F10008039002013B50C464FF6FF7301226946F5
:106F20000248FCF7ADFC00981CBD00000C060020D8
:106F30002DE9F04DC84A002490B0914205DA21F0C5
:106F40000043934201D805D120B110B0BDE8F04D07
:106F5000FEF7D4BDB1F5801F1BDA53EA000209D059
:106F6000002911DA0120FEF7E1FD10B0BDE8F04D77
:106F7000FEF7C7BD0220FEF7D9FDFEF7B7FD10B042
:106F800081F00041BDE8F08D6FF035043622F9F74D
:106F900067FD04EB2152C1F31308B049A2F2FF339D
:106FA000414401F4801282F07F6103EB225281F0B0
:106FB0004051009241EA08010022A94BF9F74AFD2D
:106FC000044608F10200A74EC0F313000D467E44AC
:106FD000032867D2D6E900232046F9F777FB1ED1B4
:106FE0000098002802BFD6E9000110B0BDE8F08D7E
:106FF000F9F79EFD07460C469B4A9C4BF9F7FEF9B4
:1070000006460D469A4A9B4B38462146F9F7F6F953
:1070100010B032462B46BDE8F04DF9F77ABC4FF080
:107020005532954B20462946F9F7E8F90022934B53
:10703000F9F713FD06460F4622462B461046194621
:10704000F9F7DCF932463B46F9F7D8F906460098DD
:107050000F46F0B1F9F76CFD80468A46824A834BB1
:10706000F9F7CCF932463B46F9F7F7FC22462B46B6
:10707000F9F7F0FC05460C467D4A7E4B40465146EA
:10708000F9F7BCF910B02A462346BDE8F04DF9F7F0
:10709000E1BC0B4610B0324620462946BDE8F04D13
:1070A000F9F7D8BC00224FF080432046F9F731FCB5
:1070B00002460B4620462946F9F712FA06460F46C5
:1070C0000098F9F735FDCDE9040132463B461046FC
:1070D0003946F9F793F90C9069480C9A40440190AD
:1070E00009910B461046F9F789F982460246654830
:1070F0008B46C8F151080B4608F5D7280321784480
:10710000FEF79FFC52465B46F9F778F90A905E4815
:107110000D9152465B4604217844FEF792FC099B90
:107120000C9AF9F76BF9844601980D9B40EA080820
:1071300060460A9AF9F7EDFB83460891B8F1000F13
:107140004EDD4FF0FF3220462946F9F789FC2246F2
:107150002B46F9F753F9804600988A4660B3DDE97B
:107160000401414A414BF9F749F9099100905A4607
:1071700040465146089BF9F7CCFB32463B46F9F7AF
:107180003DF9099B009AF9F7C4FB42465346F9F7CB
:1071900064FC22462B46F9F75DFC04460D46DDE90A
:1071A0000401334A334BF9F729F910B022462B4634
:1071B000BDE8F04DF9F74EBC5A464046089BF9F73A
:1071C000A8FB32463B46F9F719F942465346F9F710
:1071D00044FC10B022462B46BDE8F04DF9F73DBC0B
:1071E000009840B3DDE904011F4A204BF9F706F986
:1071F00080468A465A4620462946089BF9F72AFCCB
:1072000032463B46F9F7FAF842465346F9F722FC74
:1072100022462B46F9F71EFC04460D46DDE9040123
:10722000134A144BF9F7EAF810B022462B46BDE892
:10723000F04DF9F70FBC0B465A4620462946F9F7A0
:1072400009FC32463B46F9F7D9F810B022462B46E6
:10725000BDE8F04DF9F701BC0000F07F645F090064
:107260000000F03F9E2C0000763C7935EF39EA3D76
:107270000000E0FE422EE63F5555D53F0000E03FBE
:1072800086EBF9FF362B0000342B00002DE9F0418E
:10729000044630480025814205DA21F0004282424E
:1072A00001D805D124B12046BDE8F041FEF726BC47
:1072B000B1F5801F1BDA52EA040008D000290FDA6A
:1072C0000120FEF733FCBDE8F041FEF71ABC0220B6
:1072D000FEF72CFCFEF70AFC81F00041BDE8F081CE
:1072E0006FF0350536222046F9F7BAFB044605EB68
:1072F0002150A0F2FF32D00F40F2FF331B1A0D468F
:1073000063F31F551044F9F713FC06460F46294650
:107310002046FFF70DFE104A104BF9F76FF80446B0
:107320000D460F4A0F4B30463946F9F767F82246AB
:107330002B46F9F7EEFA05460C460B4A0B4B304646
:107340003946F9F75BF82A462346BDE8F041F9F7DC
:10735000E0BA00000000F07F0EE526157BCBDB3F96
:10736000362BF111F3FE593D00609F501344D33F7B
:10737000FAF7B6FFFDF7D3FDFCF79EFCFCF782FCA5
:10738000FCF7C8FBFCF786FDFCF730FDFCF7D8FDE9
:10739000FCF718FEFCF784FEFCF79EFE00200A496D
:1073A0000968486300210848FCF720F900F024F838
:1073B000064A0021064800F065F80649086000F01A
:1073C00031F800BFFEE700007C0500208C99000822
:1073D000D94E00082001002070B50546FEF72EFBAF
:1073E00010B16FF0050404E0002415B1284601F047
:1073F000C5F8204670BD000010B5FEF71FFB10B1A8
:107400006FF0050409E00648006820B9012004492E
:107410000860002401E04FF0FF34204610BD00005A
:10742000DC01002070B5FEF709FB10B16FF0050418
:107430001FE011480068012819D100BF801F0021FA
:10744000002804DB0A07130E0C4A135406E00A074F
:10745000150E0B4A00F00F031B1FD55400BF00BFD1
:1074600002200549086001F069F9002401E04FF0AD
:10747000FF34204670BD0000DC01002000E400E085
:1074800018ED00E02DE9FF478046894614460020AC
:107490000390FEF7D3FA00284ED1B8F1000F4BD07D
:1074A000802618258246471E44B3206808B1D4F8C8
:1074B00000A0A06900B1A5692DB1382D03D82079AD
:1074C00000F0010018B1002004B0BDE8F087606949
:1074D00008B160698608A06840B1E0685C2805D3FF
:1074E000206918B1606908B1012708E0A06830B9C7
:1074F000E06820B9206910B9002700E00027012FBB
:107500000CD12169A0684B463246CDE9005102906A
:107510005146404601F04EFF03900DE067B903A8C5
:10752000B2B24B465146CDE90050404601F010FF43
:10753000012801D0002003900398C5E72DE9F04110
:1075400005460E461648076816480068001D00F0FC
:107550002BFE681C38B936B112480168091D124863
:1075600000F078FE1AE07C190E4800684460BC42C6
:1075700007D20C480168091D0C48006800F050FE55
:107580000CE008480168091D0948006800F048FE41
:1075900008480068844201D206480460BDE8F081D2
:1075A000A00100208C0100207C120020940100200A
:1075B00090010020BC01002010B5044600F0B8FE88
:1075C00024480068401C234908602348006840B9EB
:1075D000214804600846006801280DD100F0FCF93C
:1075E0000AE01E48006838B91B480068C06AE16AB2
:1075F000884201D81848046019480068401C18499E
:1076000008600846006860641649E06A09688842B4
:1076100002D91449E06A0860E16A01EB8101124A6B
:1076200002EB8100211D00F015FE00F0ABFE0B48BF
:10763000006868B108480068C06AE16A884207D2F9
:107640004FF0805009490860BFF34F8FBFF36F8F31
:1076500010BD00009C0100208C010020A80100202A
:10766000B8010020A4010020CC0D002004ED00E0B2
:1076700008B500F05DFE12480068E8B9114800F056
:10768000BFFD114800F0BCFD0E48104908600E48CF
:107690000F49086000200F4B0F4A102100900A206C
:1076A00001F04EFB064908600846006820B10BA1B6
:1076B0000348006800F026FF00F064FE08BD0000EB
:1076C000D001002090120020A4120020C801002048
:1076D000CC010020B812002008130020546D725114
:1076E0000000000010B516E000F022FE0C48C06853
:1076F000C468201D00F058FD0A480068401E094972
:10770000086009480068401E0749086000F03AFE1A
:10771000204600F05FF8044800680028E4D110BD5E
:10772000681200209C0100209801002070B50446DA
:107730000D46206C70B1216CE0680144E160D4E931
:107740000210884201D32168E1602846226CE1687A
:10775000F8F768FD70BD2DE9F04104460F46154667
:107760004FF00008A66B206C48B9206800282CD187
:10777000A06801F035FF80460020A06025E07DB9BB
:107780003946226C6068F8F74DFD216C606808444A
:107790006060D4E90101884217D32068606014E07A
:1077A0003946226CE068F8F73DFD216CE068411A2B
:1077B000E1602168E068884203D2216CA068411A28
:1077C000E160022D01D106B1761E701CA063404617
:1077D000BDE8F08110B5044694F8590030B9206B2B
:1077E00000F0EEFD204600F0EBFD1AE094F85900A1
:1077F000012803D1204600F0E3FD12E094F859007F
:10780000022801D1012000E0002050B900BF502023
:1078100080F31188BFF34F8FBFF36F8F00BF00BF9E
:10782000FEE710BD0146084A126812680AB9012233
:1078300000E000220A600A6822B9034A1268D2688E
:10784000106800E000207047C801002030B54FF4F8
:10785000F053174800F007042CB1C01D20F00700BA
:10786000134C041B1B1B0246124C22600024114DBA
:107870006C60D018083820F007000F4C20600024FE
:107880000D4D2D686C600C4D2D682C601146441A0E
:107890004C60094C24680C60084D4C682C60084D05
:1078A0004C682C604FF00044064D2C6030BD000049
:1078B000601A0020E0010020E8010020F001002013
:1078C000EC010020FC01002000BFFFF70BFF064881
:1078D00000680128F9D94FF0805004490860BFF3CF
:1078E0004F8FBFF36F8FF0E7CC0D002004ED00E069
:1078F0002DE9F04106460D4617469846069C0DB9FF
:10790000246000E02760E66325640121204601F041
:1079100087FA84F84C80BDE8F0812DE9F05F82465B
:107920000E4690469B460A9F0C9C4FEA8801A52272
:10793000206BF8F789FCA8F10100216B01EB8009AD
:1079400029F0070909F0070008B9012000E000202C
:1079500050B900BF502080F31188BFF34F8FBFF3A1
:107960006F8F00BF00BFFEE786B1002507E0715DA5
:1079700004F134004155705D00B902E06D1C102D1A
:10798000F5D300BF00214320015502E0002084F818
:107990003400382F00D33727E762E76400202065E2
:1079A000201D00F03AFC04F1180000F036FC2461C0
:1079B000C7F13800A06164620020606584F8580057
:1079C0005A465146484600F09BFB20600B9808B190
:1079D0000B980460BDE8F09F10B5002407E004EBAD
:1079E00084010F4A02EB810000F00AFC641C382C71
:1079F000F5D30C4800F004FC0B4800F001FC0B48E8
:107A000000F0FEFB0A4800F0FBFB0A4800F0F8FB20
:107A100004480949086004480849086010BD00008E
:107A2000CC0D00202C120020401200205412002007
:107A3000681200207C120020900100209401002098
:107A400010B50146164800E0006803688B42FBD37E
:107A50000246436813448B4204D143684C68234474
:107A6000436001460A464B6813440468A34211D19F
:107A70000C4C03682468A34208D04B68046864680F
:107A800023444B6003681B680B6005E0054B1B68D3
:107A90000B6001E003680B60884200D0016010BDFC
:107AA000E0010020E80100202DE9F04104460D46E8
:107AB00016461F464FF0000865602461B5420CD899
:107AC000F01BA169884202D34FF0010811E0211D8B
:107AD0000948006800F0A4FB0BE0BE4204D2BD429E
:107AE00002D34FF0010804E0211D0448006800F0B3
:107AF00097FB4046BDE8F081CC010020C801002082
:107B000070B5054600F014FCA86B08B9012400E02C
:107B1000002400F037FC204670BD70B5054600F02B
:107B200007FCA86BE96B884201D1012400E0002426
:107B300000F028FC204670BDF8B505460F461A48EF
:107B40000068C068C468201D00F02EFB94F828006F
:107B500000F00400E8B1A06941192B463A462046DE
:107B6000FFF7A2FFD8B1002003462A460146009045
:107B7000204601F091FE064656B900BF502080F322
:107B80001188BFF34F8FBFF36F8F00BF00BFFEE7B9
:107B900005E094F8280020F0010084F82800204631
:107BA000216A8847F8BD0000C8010020F0B587B001
:107BB000A0E00398002811DA04AE56B900BF5020A7
:107BC00080F31188BFF34F8FBFF36F8F00BF00BFEB
:107BD000FEE7D6E90020B168904700BF039800286F
:107BE000E6DB059C606908B9012000E0002010B9BF
:107BF000201D00F0D9FA02A800F0DEF8054603982F
:107C00000A2875D2DFE800F0090507394163060844
:107C10003A4200BF00BF00BF00BF94F8280040F008
:107C2000010084F828000498A269811803462A46B6
:107C30002046FFF739FFF8B12046216A884794F8BB
:107C4000280000F00400B8B1002000900498A16959
:107C5000421800231946204601F01EFE074657B978
:107C600000BF502080F31188BFF34F8FBFF36F8F99
:107C700000BF00BFFEE700BF3BE000BF94F8280054
:107C800020F0010084F8280033E000BF94F82800B9
:107C900040F0010084F828000498A061A06908B1B0
:107CA000012000E0002050B900BF502080F311886F
:107CB000BFF34F8FBFF36F8F00BF00BFFEE7A06918
:107CC00041192B462A462046FFF7EEFE11E094F8B4
:107CD000280000F0020018B9204600F071FB05E012
:107CE00094F8280020F0010084F8280001E0FFE764
:107CF00000BF00BF002203A90448006801F02EFA6B
:107D000000287FF456AF07B0F0BD0000D00100207E
:107D1000F8B505460C4600F06DFD684600F04CF8DD
:107D20000646009820BB44B9B54206D801F0F6FCDF
:107D300031462846FFF700FF1CE03CB10E480068C2
:107D4000006808B9012000E000200446A91B224673
:107D50000A48006800F0ECFB01F0E0FC50B94FF07D
:107D6000805007490860BFF34F8FBFF36F8F01E06A
:107D700001F0D4FCF8BD0000CC010020D0010020AF
:107D800004ED00E00A490968096809B9012100E029
:107D9000002121B14FF0FF31064A116006E004498D
:107DA0000968C968C868034A4168116070470000E3
:107DB00090010020BC01002070B5044601F068FB72
:107DC000054607480068854204D200F00BF8012000
:107DD000206001E00020206001480560284670BD59
:107DE000D80100202DE9F84334E025480068C06838
:107DF000056823480068C068C468201D00F0D4F9F5
:107E00002046216A884794F8280000F0040008B34F
:107E1000A0694619AE4207D966602461211D184841
:107E2000006800F0FDF915E0002003462A460146EF
:107E30000090204601F030FD074657B900BF5020A2
:107E400080F31188BFF34F8FBFF36F8F00BF00BF68
:107E5000FEE700BF0A480068006808B9012000E09A
:107E600000200028C1D00648D0F8008005480068EE
:107E7000034908600348C0F80080BDE8F8830000AB
:107E8000C8010020CC0100200E480068401C08B941
:107E9000012000E0002050B900BF502080F311887D
:107EA000BFF34F8FBFF36F8F00BF00BFFEE700BF70
:107EB000502080F31188BFF34F8FBFF36F8F00BF47
:107EC00000BFFEE70002002008B500BF6846FFF7CC
:107ED000A9FC044620460099FFF71AFFFFF766FE4B
:107EE000F4E770B5044600F023FA94F9455010E029
:107EF000606A08B9012000E0002038B904F12400CC
:107F000001F0C0FB18B100F0D7FB00E003E0681EF1
:107F100045B2002DECDC00BFFF2084F8450000F0E6
:107F200031FA00F005FA94F9445010E0206908B9DC
:107F3000012000E0002048B904F1100001F0A2FB8C
:107F400008B100F0B9FB681E45B200E001E0002D69
:107F5000ECDC00BFFF2084F8440000F013FA70BD91
:107F6000014621B1012904D0072906D103E00020F0
:107F700005E0022003E0062001E0042000BF00BF6E
:107F80007047000010B502480068804710BD00002F
:107F90003C02002010B502480068804710BD000078
:107FA0003402002010B502480068804710BD000070
:107FB000380200202DE9F04104464FF0000800F09F
:107FC00019FC4948006808B9FFF740FC47480068B9
:107FD0002040002870D1D4B1083404F00700B0B1BB
:107FE00004F00700C0F10800044404F0070008B9D9
:107FF000012000E0002050B900BF502080F311881C
:10800000BFF34F8FBFF36F8F00BF00BFFEE7002CA1
:1080100052D03748006884424ED8364E3046056804
:1080200001E02E462D686868A04202D22868002828
:10803000F7D12D48006885423ED0306800F108082D
:10804000286830606868001B102819D92F1907F0BC
:10805000070008B9012000E0002050B900BF5020FF
:1080600080F31188BFF34F8FBFF36F8F00BF00BF46
:10807000FEE76868001B78606C603846FFF7E0FC3C
:108080001B4968680968081A1949086008460068A9
:1080900019490968884203D21548006816490860E2
:1080A000124968680968084368600020286013481E
:1080B0000068401C1149086001F030FB08F007001F
:1080C00008B9012000E0002050B900BF502080F323
:1080D0001188BFF34F8FBFF36F8F00BF00BFFEE764
:1080E0004046BDE8F0810000E8010020FC010020CE
:1080F000EC010020E0010020F0010020F40100204C
:10810000001F4FF080730360001F21F00103036024
:10811000001F034B036014380260203870470000D2
:10812000897E00082DE9F04106460F46F8F7AFFCBE
:10813000041E0D4618BF0120284320F00040C0F166
:108140007F6000F1E040C00F0ED0301C18BF01204E
:10815000384320F00040C0F17F6000F1E040C00FE4
:1081600004BF0120FDF7E2FC20462946BDE8F0816E
:1081700070B502460C46FF25FF2309E012F8010BFB
:1081800080EA03010648405C80EA05030548455C37
:10819000201EA4F10106B4B2F0D143EA052070BD5F
:1081A000149A0008149B000801460A69D1E90130BD
:1081B0009860D1E9010358605068884201D188680D
:1081C0005060002008611068401E10601068704701
:1081D000034B0360034B0B60802313607047000068
:1081E000A813002004140020034B0360034B0B6012
:1081F0004FF480731360704704160020601600204F
:1082000000F1080141604FF0FF31816000F1080189
:10821000C160016100210160704700210161704768
:1082200010B502460B685C1C0CB9106907E002F13E
:10823000080000E04068446824689C42FAD9446819
:108240004C604C68A160886041600A611468641CDD
:10825000146010BD42684A6093688B6093685960EF
:108260009160086103685B1C0360704700B50346BA
:108270000A4633B11148008840F020000F490880B9
:1082800005E00E48008820F020000C49088042B12B
:10829000FBF71CFC0948008840F080000749088073
:1082A0000AE00648008820F080000449088008465B
:1082B000008840F04000088000BD00000C380140FC
:1082C0000C48008820F001000A4908800020094974
:1082D0002431088007480C30008820F0010005494F
:1082E0000C310880081D008820F00100091D08805D
:1082F00070470000001400400C48008820F0010086
:108300000A490880081F008840F00100091F088002
:10831000002006491431088004481038008840F0D5
:108320000100024910390880704700001014004015
:1083300000BF502080F31188BFF34F8FBFF36F8FC2
:1083400000BF0E480068401C0C49086008460068E1
:10835000012812D10A480068C0B208B9012000E023
:10836000002050B900BF502080F31188BFF34F8F19
:10837000BFF36F8F00BF00BFFEE770470002002011
:1083800004ED00E00D48006850B900BF502080F3B4
:108390001188BFF34F8FBFF36F8F00BF00BFFEE7A1
:1083A00006480068401E054908600846006820B974
:1083B000002080F3118800BF00BF7047000200203A
:1083C00070B506463546002E44D0083D2C4622495D
:1083D00060680968084008B1012000E0002050B939
:1083E00000BF502080F31188BFF34F8FBFF36F8F12
:1083F00000BF00BFFEE7206808B9012000E00020B0
:1084000050B900BF502080F31188BFF34F8FBFF3E6
:108410006F8F00BF00BFFEE70F4960680968084022
:10842000C0B12068B0B90C496068096888436060D1
:1084300000F0E0F9094960680968084407490860E4
:108440002046FFF7FDFA06480068401C0449086012
:1084500001F064F970BD0000FC010020EC01002077
:10846000F801002000204FF0E021086188610648F3
:1084700000684FF47A71B0FBF1F0401E4FF0E0213C
:1084800048610720086170478801002070B5F7F740
:10849000A3FE0446102C16D304F1E02090F8F0530C
:1084A00015480078854201DB012000E0002050B92A
:1084B00000BF502080F31188BFF34F8FBFF36F8F41
:1084C00000BF00BFFEE70D48006800F4E0600C4903
:1084D0000968884201D8012000E0002050B900BF9F
:1084E000502080F31188BFF34F8FBFF36F8F00BF11
:1084F00000BFFEE770BD0000040200200CED00E0AC
:1085000008020020024600200BE0084B53F83030F0
:1085100033B9064B43F8301003EBC0035A6002E056
:10852000401C0828F1D300BF704700008C0D0020CC
:108530002DE9F04105460E4617462C46FFF7F8FE9A
:1085400094F94400401C10B9002084F8440094F9C8
:108550004500401C10B9002084F84500FFF712FFC9
:10856000A06B28B93A46314604F1240000F0C6F861
:108570002046FFF7B6FCBDE8F081000070B5044668
:108580000025D4B11248006808B9012000E000209D
:1085900050B900BF502080F31188BFF34F8FBFF355
:1085A0006F8F00BF00BFFEE700F024F900212046D6
:1085B000FEF7C4FF01F0B2F805463DB94FF0805018
:1085C00004490860BFF34F8FBFF36F8F70BD000089
:1085D000C401002004ED00E070B50546FFF7A8FED9
:1085E00015B92748006800E028460446201DFFF71B
:1085F000DBFDA06A18B104F11800FFF7D5FD214892
:108600000068401C1F4908601D480068844209D169
:10861000211D1D48FFF71EFE1C480068401C1B4919
:10862000086009E01A480068401E194908602046A1
:10863000FFF7D0F8FFF7A6FBFFF7A4FE1548006888
:10864000E8B10F480068844219D11348006808B99E
:10865000012000E0002050B900BF502080F31188B5
:10866000BFF34F8FBFF36F8F00BF00BFFEE74FF028
:1086700080500A490860BFF34F8FBFF36F8F70BD02
:108680008C010020B8010020681200209801002011
:108690009C010020A8010020C401002004ED00E09E
:1086A0000349096801600349096841607047000097
:1086B000B4010020A001002001200149086070479A
:1086C000B001002070B504460D4654B900BF5020DB
:1086D00080F31188BFF34F8FBFF36F8F00BF00BFD0
:1086E000FEE70548016818312046FFF799FD012192
:1086F0002846FEF723FF70BD8C01002070B50546AB
:108700000E46144655B900BF502080F31188BFF3C0
:108710004F8FBFF36F8F00BF00BFFEE706480168B1
:1087200018312846FFF796FD0CB14FF0FF36214671
:108730003046FEF703FF70BD8C01002010B586B0F7
:1087400000200590049003AA04A905A8FFF740FDA6
:108750000022DDE904101346CDE9002102901EA19C
:108760001F48039A00F026FE1E490860084600686C
:1087700008B1012400E00024012C02D101F050F8DE
:108780000446012C15D100BF502080F31188BFF39F
:108790004F8FBFF36F8F00BF4FF0FF30124908605B
:1087A00001201249086000201149086000F032FAE7
:1087B00010E0601C08B1012000E0002050B900BFAB
:1087C000502080F31188BFF34F8FBFF36F8F00BF2E
:1087D00000BFFEE706B010BD49444C450000000054
:1087E000C9780008C0010020BC010020A8010020B9
:1087F000A001002002480068401C01490860704741
:10880000C40100201E48006818B101201D490860FD
:1088100034E000201B4908601B4801680CE051B996
:1088200000BF502080F31188BFF34F8FBFF36F8FCD
:1088300000BF00BFFEE7491E01EB8100134A52F85A
:10884000200008B9012000E000200028E7D101EB5A
:1088500081020E4B03EB820042685268426000F1D5
:1088600008024368934202D14268526842604268FB
:10887000D268074B1A600448016000BF70470000CF
:10888000C4010020B0010020A4010020CC0D002074
:108890008C01002001460020054A127832B1054AB9
:1088A00012780A700022024B1A70012070470000F3
:1088B000D5020020D40200200020024908700120C7
:1088C00070470000D502002001460120024A1070C6
:1088D0000248017001207047D5020020D402002018
:1088E00010B50446FBF7DCF8024800882070012030
:1088F00010BD0000043801402DE9F04107460C4648
:1089000015461E463548806940F0040033498861A9
:10891000334800686FF30B0000F2B3403049086041
:108920002E48806940F480402C498861FBF7B8F8F4
:1089300000202C490880091D0880091D08800C2092
:108940002849088028480068B0FBF4F0091F088017
:10895000082D02D0092D0ED106E02248008820F40F
:1089600080502049088006E01E48008840F480506E
:108970001C49088000BF00BF26B1012E09D0022E7D
:108980001FD112E01748008820F480601549088044
:1089900017E01448008840F4007012490880084627
:1089A000008840F4806008800BE00E48008820F4C6
:1089B00000700C4908800846008840F480600880F8
:1089C00000BF00BF0748008840F4005005490880F8
:1089D0002520FDF709F80120BDE8F08100100240D4
:1089E000040801400C3801408801002000B502460F
:1089F000FBF76CF801480280012000BD04380140FB
:108A000010B504461048C06940F020000E49C86106
:108A100000200E4908800E4800684CF25031B0FB2F
:108A2000F1F0401E094928310880081D048001200A
:108A300006491431088005490C3108803720FCF7BD
:108A4000D3FF012010BD00000010024000140040C0
:108A50008801002038B500246846FFF741FF1C4814
:108A6000007830B101280AD0022819D003282BD170
:108A700002E0FFF741FC27E0FFF73EFC24E0002086
:108A8000144908809DF800200888411C114B19806A
:108A900011490A5402200E490870FFF72DFC13E01B
:108AA0000C480088FF2809DC9DF800200949088847
:108AB000411C084B198008490A5402E0032004496C
:108AC0000870FFF719FC00BF00BF204638BD00004A
:108AD000110200201A0200208038002010B5002466
:108AE0000D48007820B1022807D003280BD109E0F7
:108AF0000020FFF7E9FE044606E00120FFF7E4FE50
:108B0000044601E000E000BF00BFFFF7D9FB0120F1
:108B100001490870204610BD1102002010B5002444
:108B20001648007810B1012824D104E0002101206A
:108B3000FFF79CFB1EE01248008878B111490968D4
:108B40000878FFF753FF0F480068401C0D49086084
:108B50000B480088401E0A4908800AE00320FFF7FE
:108B6000B3FE044600210120FFF780FB00200349EB
:108B7000087000BF00BF204610BD0000100200209A
:108B80001802002014020020F0B503460C461546DA
:108B9000E208A4EBC20087B20120A840401E86B2C2
:108BA000995C501C185C41EA002139413140C8B23F
:108BB000F0BD2DE9F043044615461F46C808A1EB59
:108BC000C0081FFA88FC07FA0CF81FFA88F74FF064
:108BD000010808FA05F8A8F101081FFA88F6A1EBC8
:108BE000C00806FA08F81FFA88F6225C00F10108AE
:108BF00014F8088042EA082222EA060848EA070236
:108C000022544FEA222900F1010804F80890BDE837
:108C1000F08300001CB53849084600780190FF2019
:108C20000A4610700846007800909DF8000000F099
:108C3000F0009DF80020904201D1012000E00020CA
:108C400050B900BF502080F31188BFF34F8FBFF39E
:108C50006F8F00BF00BFFEE79DF8000000F05000DE
:108C6000264A10700720264A106009E02448006850
:108C7000401E234A10609DF800004006000E009040
:108C80009DF8000000F080008028EFD01C480068AC
:108C9000C0F10700042801D1012000E0002050B9F4
:108CA00000BF502080F31188BFF34F8FBFF36F8F49
:108CB00000BF00BFFEE7124800680002104A1060C3
:108CC0001046008800F4E06010600B4A01981070B4
:108CD0000C48006840F470000A49086008460068C3
:108CE00040F070400860FFF7BDFB002006490860B7
:108CF000F7F73CFA00201CBD00E400E0040200206D
:108D00000802002020ED00E00002002010B500BFA6
:108D1000502080F31188BFF34F8FBFF36F8F00BFD8
:108D200000F0BCFB18B14FF080500449086000BF50
:108D3000002080F3118800BF10BD000004ED00E0AA
:108D40002DE9F84380460E4617461D46DDF8209073
:108D5000B8F1000F01D0012000E0002050B900BFA1
:108D6000502080F31188BFF34F8FBFF36F8F00BF88
:108D700000BFFEE70DB1012000E0002050B900BFA8
:108D8000502080F31188BFF34F8FBFF36F8F00BF68
:108D900000BFFEE707B10EB1012000E0002050B98E
:108DA00000BF502080F31188BFF34F8FBFF36F8F48
:108DB00000BF00BFFEE707B90EB9012000E00020A8
:108DC00050B900BF502080F31188BFF34F8FBFF31D
:108DD0006F8F00BF00BFFEE7502000900098502822
:108DE00001D1012000E0002050B900BF502080F3E5
:108DF0001188BFF34F8FBFF36F8F00BF00BFFEE737
:108E000000BF2C464CB1012084F846004B463A4640
:108E1000314640460094FEF76BFD2046BDE8F883DE
:108E200070B505460E462C4654B900BF502080F35D
:108E30001188BFF34F8FBFF36F8F00BF00BFFEE7F6
:108E4000FFF776FAD4E90F12206801FB0200A06058
:108E50000020A06320686060E06B401E226C2168E7
:108E600000FB0211E160FF2084F8440084F8450013
:108E70009EB9206908B9012000E00020A8B904F1DA
:108E8000100000F0FFFB80B14FF0805009490860EE
:108E9000BFF34F8FBFF36F8F07E004F11000FFF7B0
:108EA000AFF904F12400FFF7ABF9FFF76BFA0120EB
:108EB00070BD000004ED00E02DE9FF4383B00646DD
:108EC00088461D464FF00009344654B900BF502073
:108ED00080F31188BFF34F8FBFF36F8F00BF00BFC8
:108EE000FEE7B8F1000F01D1206C08B9012000E0C5
:108EF000002050B900BF502080F31188BFF34F8F7E
:108F0000BFF36F8F00BF00BFFEE7022D02D1E06B01
:108F1000012801D1012000E0002050B900BF5020FD
:108F200080F31188BFF34F8FBFF36F8F00BF00BF77
:108F3000FEE700F09DFA08B9059808B9012000E0A5
:108F4000002050B900BF502080F31188BFF34F8F2D
:108F5000BFF36F8F00BF00BFFEE700BFFFF7E8F968
:108F6000A06BE16B884201D3022D28D12A464146ED
:108F70002046FEF7F0FB0746606A08B9012000E0D2
:108F8000002068B904F1240000F07CFB88B14FF0A8
:108F9000805032490860BFF34F8FBFF36F8F08E0F6
:108FA0003FB14FF080502D490860BFF34F8FBFF3A2
:108FB0006F8FFFF7E7F9012007B0BDE8F083059850
:108FC00018B9FFF7DFF90020F6E7B9F1000F04D177
:108FD00001A8FFF765FB4FF00109FFF7D3F9FFF791
:108FE00009FCFFF7A5F994F94400401C10B90020D2
:108FF00084F8440094F94500401C10B9002084F81E
:109000004500FFF7BFF905A901A800F05BF9F0B929
:109010002046FEF782FDA0B104F110000599FFF78C
:1090200051FB2046FEF75DFF00F078FB002895D14C
:109030004FF0805009490860BFF34F8FBFF36F8F27
:109040008CE72046FEF74DFF00F068FB86E72046E0
:10905000FEF747FF00F062FB0020ADE704ED00E003
:109060002DE9F84F07468A4690461E463C4654B9BD
:1090700000BF502080F31188BFF34F8FBFF36F8F75
:1090800000BF00BFFEE7BAF1000F01D1206C08B9A4
:10909000012000E0002050B900BF502080F311886B
:1090A000BFF34F8FBFF36F8F00BF00BFFEE7022EED
:1090B00002D1E06B012801D1012000E0002050B96D
:1090C00000BF502080F31188BFF34F8FBFF36F8F25
:1090D00000BF00BFFEE7FFF7D9F900BF5021EFF353
:1090E000118081F31188BFF34F8FBFF36F8F00BFE3
:1090F0000546A06BE16B884201D3022E25D194F97D
:1091000045B0A06B0090324651462046FEF723FB47
:109110000BF1010088B9606A08B9012000E0002065
:1091200050B904F1240000F0ADFA28B1B8F1000FF5
:1091300002D00120C8F8000004E00BF1010040B2A9
:1091400084F845004FF0010901E04FF0000900BF2D
:1091500085F3118800BF4846BDE8F88F2DE9F74137
:1091600083B005460E464FF000082C4654B900BFA8
:10917000502080F31188BFF34F8FBFF36F8F00BF74
:1091800000BFFEE70EB9206C08B9012000E0002006
:1091900050B900BF502080F31188BFF34F8FBFF349
:1091A0006F8F00BF00BFFEE700F062F908B90598B5
:1091B00008B9012000E0002050B900BF502080F322
:1091C0001188BFF34F8FBFF36F8F00BF00BFFEE763
:1091D00000BFFFF7ADF8A76BF7B131462046FEF7A9
:1091E000A5FA781EA063206908B9012000E00020DC
:1091F00060B904F1100000F045FA38B14FF080502A
:109200002F490860BFF34F8FBFF36F8FFFF7BAF896
:10921000012006B0BDE8F081059818B9FFF7B2F853
:109220000020F6E7B8F1000F04D101A8FFF738FAE3
:109230004FF00108FFF7A6F8FFF7DCFAFFF778F820
:1092400094F94400401C10B9002084F8440094F9BB
:109250004500401C10B9002084F84500FFF792F843
:1092600005A901A800F02EF8F0B92046FEF748FC49
:10927000A0B104F124000599FFF724FA2046FEF777
:1092800030FE00F04BFA0028A3D14FF080500C497B
:109290000860BFF34F8FBFF36F8F9AE72046FEF74A
:1092A00020FE00F03BFA94E72046FEF71AFE00F09D
:1092B00035FA2046FEF724FC00288AD00020A8E7D3
:1092C00004ED00E070B505460C4655B900BF5020CE
:1092D00080F31188BFF34F8FBFF36F8F00BF00BFC4
:1092E000FEE754B900BF502080F31188BFF34F8FC1
:1092F000BFF36F8F00BF00BFFEE7FFF719F81248FA
:1093000002686868131A2068401C08B9002617E034
:109310000E4928680968884204D06868904201D8DC
:1093200001260DE02068984207D92068C01A206005
:109330002846FFF7B5F9002602E00020206001264C
:10934000FFF720F8304670BDA0010020B4010020D6
:109350002DE9FF4F85B0804689461746DDE912ABFF
:10936000B800FEF727FE064656B15C20FEF722FE47
:1093700004460CB1266304E03046FFF721F800E014
:1093800000248CB1002084F85900CDE900ABCDE970
:1093900002403A4649464046089BFEF7BEFA204640
:1093A000FEF70AF9012501E04FF0FF35284609B024
:1093B000BDE8F08F2DE9F04F85B00746884691460D
:1093C0009A46DDE90EB6109C0EB1012000E00020A7
:1093D00050B900BF502080F31188BFF34F8FBFF307
:1093E0006F8F00BF00BFFEE70CB1012000E000203E
:1093F00050B900BF502080F31188BFF34F8FBFF3E7
:109400006F8F00BF00BFFEE75C20039003985C28CD
:1094100001D1012000E0002050B900BF502080F3AE
:109420001188BFF34F8FBFF36F8F00BF00BFFEE700
:1094300000BFB4B1AEB125462C462E63022085F89C
:109440005900002004A953464A46CDE900B1CDE9B0
:10945000025041463846FEF760FA2846FEF7ACF85F
:1094600001E000200490049805B0BDE8F08F0000F2
:109470000549096809B9012005E00449096809B9E5
:10948000022000E000207047A8010020C401002055
:109490000149086870470000A00100202DE9F04153
:1094A0004FF000084348006800287BD1424800681C
:1094B000451C4148056015BB40480068006808B974
:1094C000012000E0002050B900BF502080F3118837
:1094D000BFF34F8FBFF36F8F00BF00BFFEE737486A
:1094E00007683748006835490860354807603548DF
:1094F0000068401C33490860FEF744FC00BF324856
:10950000006885423BD300BF2C480068006808B95A
:10951000012000E0002020B14FF0FF302A49086010
:109520002CE026480068C068C4686668B54202D26C
:109530002548066022E0201DFEF736FEA06A18B11D
:1095400004F11800FEF730FE2049E06A09688842FD
:1095500002D91E49E06A0860E16A01EB81011C4AF8
:1095600002EB8100211DFEF775FE1A49E06A0968C9
:10957000C96A8842C8D34FF00108C5E700BF154843
:109580000068C06A00EB8000114951F820000128F2
:1095900001D94FF001081048006808B14FF00108E8
:1095A00005E0FFE70D480068401C0C490860404694
:1095B000BDE8F081C4010020A0010020900100203E
:1095C00094010020B4010020BC010020A40100206F
:1095D000CC0D00208C010020B0010020AC01002047
:1095E00070B505462C460026002D43D02248006861
:1095F000844201D1012000E0002050B900BF50207A
:1096000080F31188BFF34F8FBFF36F8F00BF00BF90
:10961000FEE7206D50B900BF502080F31188BFF3E2
:109620004F8FBFF36F8F00BF00BFFEE7206D401E5E
:109630002065E16CE06A88421CD0206DD0B9201D05
:10964000FEF7B2FDE06CE062E06AC0F13800A061B4
:109650000A49E06A0968884202D90849E06A086054
:10966000E16A01EB8101064A02EB8100211DFEF750
:10967000F1FD0126304670BD8C010020A4010020C0
:10968000CC0D002070B50646F068C46854B900BF20
:10969000502080F31188BFF34F8FBFF36F8F00BF4F
:1096A00000BFFEE704F11800FEF77EFD15480068D4
:1096B000A0B9201DFEF778FD1349E06A09688842C9
:1096C00002D91149E06A0860E16A01EB81010F4AA1
:1096D00002EB8100211DFEF7BDFD04E004F118013D
:1096E0000B48FEF7B7FD0B49E06A0968C96A884272
:1096F00004D9012501200849086000E0002528461A
:1097000070BD0000C4010020A4010020CC0D002089
:10971000541200208C010020B001002070B50024FC
:1097200000263648006850B900BF502080F31188E9
:10973000BFF34F8FBFF36F8F00BF00BFFEE7FEF791
:10974000F7FD2E480068401E2C4908600846006856
:1097500000284ED12A48006800284AD023E0294832
:10976000C068C46804F11800FEF71EFD201DFEF756
:109770001BFD2549E06A0968884202D92249E06A4E
:109780000860E16A01EB8101204A02EB8100211DA2
:10979000FEF760FD1E49E06A0968C96A884202D383
:1097A00001201C4908601748006808B9012000E042
:1097B00000200028D3D00CB1FEF7E4FA1648056863
:1097C00065B100BFFFF76AFE10B1012011490860C2
:1097D0006D1E002DF6D100200F4908600D4800686D
:1097E00038B1012630070D490860BFF34F8FBFF332
:1097F0006F8FFEF7C7FD304670BD0000C40100202A
:109800009C01002054120020A4010020CC0D002057
:109810008C010020B0010020AC01002004ED00E02C
:1098200010B586B00024FDF723FF16480068D0B1BC
:1098300000200590049003AA04A905A8FEF7D4FC13
:109840000222DDE904100023CDE9002102900EA1DF
:109850000F48039AFFF7AEFD0E49086008460068FE
:1098600000B1012400BF54B900BF502080F311881B
:10987000BFF34F8FBFF36F8F00BF00BFFEE72046DF
:1098800006B010BDD0010020546D722053766300E5
:10989000C97E0008D40100202DE9FF4704460D468B
:1098A00016461F46DDF830804FF0000954B900BF5E
:1098B000502080F31188BFF34F8FBFF36F8F00BF2D
:1098C00000BFFEE71448006810B3009501960294AB
:1098D000062D15DAFFF7CCFD022808D100234246F9
:1098E00069460D480068FFF7E7FA814610E000235B
:1098F0001A46694608480068FFF7DEFA814607E025
:1099000000233A46694604480068FFF7A9FB8146F0
:10991000484604B0BDE8F087D00100201450000094
:10992000E8FD000048E80100000000000000000021
:1099300000000000000000000000C8420080BB449E
:109940000080BB4400000000000000000000000098
:109950000000000000401C4600409C4500409C4622
:1099600000000000000000000000000000000000F7
:109970000000204100007A4400007A44000000000A
:10998000000000000000000000000000789C0008BB
:1099900000000000000000000000000000000000C7
:1099A000000300001800000000000000000000009C
:1099B00008000019849C000800000000000000005E
:1099C000000000000000000000020000180000007D
:1099D000000000000000000002030405060708095B
:1099E0000A0B0C0D0E0F10100102020304050607EE
:1099F00008090A0B0C0D0E0F1010010200000000E8
:109A0000000000000102030406070809000000002E
:109A10000102030400C1814001C0804101C08041B6
:109A200000C1814001C0804100C1814000C181402E
:109A300001C0804101C0804100C1814000C181401E
:109A400001C0804100C1814001C0804101C080410E
:109A500000C1814001C0804100C1814000C18140FE
:109A600001C0804100C1814001C0804101C08041EE
:109A700000C1814000C1814001C0804101C08041DE
:109A800000C1814001C0804100C1814000C18140CE
:109A900001C0804101C0804100C1814000C18140BE
:109AA00001C0804100C1814001C0804101C08041AE
:109AB00000C1814000C1814001C0804101C080419E
:109AC00000C1814001C0804100C1814000C181408E
:109AD00001C0804100C1814001C0804101C080417E
:109AE00000C1814001C0804100C1814000C181406E
:109AF00001C0804101C0804100C1814000C181405E
:109B000001C0804100C1814001C0804101C080414D
:109B100000C1814000C0C101C30302C2C60607C71D
:109B200005C5C404CC0C0DCD0FCFCE0E0ACACB0B8D
:109B3000C90908C8D81819D91BDBDA1A1EDEDF1FBD
:109B4000DD1D1CDC14D4D515D71716D6D21213D3AD
:109B500011D1D010F03031F133F3F23236F6F7375D
:109B6000F53534F43CFCFD3DFF3F3EFEFA3A3BFB4D
:109B700039F9F83828E8E929EB2B2AEAEE2E2FEFFD
:109B80002DEDEC2CE42425E527E7E62622E2E3236D
:109B9000E12120E0A06061A163A3A26266A6A7679D
:109BA000A56564A46CACAD6DAF6F6EAEAA6A6BAB0D
:109BB00069A9A86878B8B979BB7B7ABABE7E7FBF3D
:109BC0007DBDBC7CB47475B577B7B67672B2B3732D
:109BD000B17170B0509091519353529296565797DD
:109BE000559594549C5C5D9D5F9F9E5E5A9A9B5BCD
:109BF00099595898884849894B8B8A4A4E8E8F4F7D
:109C00008D4D4C8C448485458747468682424383EC
:109C100041818040949C000800000000000000008A
:109C20000000000000000000000500002800000007
:109C3000000000000000000004FA97999999D93FAC
:109C4000AF788E1DC571CC3F9FC678D0099AC33FAF
:109C5000935555555555E53F599322942449D23F84
:109C6000DE03CB966446C73F44523EDF12F1C23F4B
:109C7000000000000000000064656661756C7454AB
:109C800061736B0053616D706C6552756E546173D6
:109C90006B0000004D4252756E5461736B00000002
:109CA000C09C000800000020EC0200001A0C000814
:109CB000509D0008EC020020EC3B00001E5B0008F9
:109CC000011A23A041137A440420409C468BF401DE
:109CD00004011023204E4BD0070401117C401C4688
:109CE00004091784290409113809161C01616974D3
:109CF000BA2CEE4264E2C85A010121C34842859A57
:109D000099993E2A1028410375127A1AAA01011A5C
:109D1000022902321113CD67330804136B6633082E
:109D20000313DF652A08E0133769330806136568F3
:109D30003308171AF72029F41385643308051AF538
:109D400038320F1AA72029721A3338015400000044
:0400000508000131BD
:00000001FF
